:0400000057EF00F0C6
:10000800025E025E025E025E025E025E025EEF5900
:10001800025E025E025E025E025E025E025E025ED8
:10002800025E025E025E025E025E025E025E025EC8
:10003800025E025E025E4F58025E025E025ED25AA5
:10004800025E025E025E025E2B00025E025E025EDD
:10005800025E025E025E025E025E025E025E025E98
:10006800025E025E025E025E025E025E025E025E88
:10007800025E025E2B00025E025E025E2B002B0017
:100088002B002B002B002B002B002B00025E025EA6
:100098004F5D025E025E025E2B002B002B002B00E0
:0A00A800025E025EFF00EBEFB0F015
:10F4A4000000000000001B1B0000181818181B1B8C
:10F4B4000000030303031B1B00001B1B1B1B1B1B64
:10F4C40000040E1F0404040400040404041F0E04B6
:10F4D400001112140B110203000E0A0E00000000AA
:10F4E400005A7701F87201767601FC51010260013D
:10F4F4008864015E5F014C7701F87701F477012895
:10F504007401A07701A877013E77019877012077ED
:10F51400019E68010665011077010080C094D42023
:10F524002000204861726477617265203A2042416C
:10F5340053452031384632374B3432202B20493260
:10F544004331204C434434783230202B20494E41FF
:10F55400323236202B20554152543120313135324C
:10F564003030202B206D6F64756C65204942542027
:10F5740032204D6F7366657420493243310D0A2081
:10F58400536368656D613A2043617274655F506FBF
:10F59400727461696C5F325F56616E746175785F15
:10F5A4003234765F482D656E2D4D4F534645545F7A
:10F5B400494E413232362D484950343038325F4654
:10F5C400515033304E30364C5F56352E302E332E5C
:10F5D40070646620627920482E542E0D0A0D0A00AC
:10F5E40020417574726573203A0D0A20204C4344FF
:10F5F4005F34626974735F4932435F323032342D51
:10F6040030312C2055415254315F46756E63746914
:10F614006F6E732E68202C206D63632E682C0D0A88
:10F624000045434F2E2E2E2E0042415252455F4735
:10F634000042415252455F440042415252454744C0
:10F6440000464C454348204800464C4543485F42E9
:10F6540000312F32486575720044454752454320B6
:10F6640000204C43445F63686172735F5370656349
:10F67400696175785F323032342E682C2020204541
:10F684006570726F6D203A20456570726F6D2E2E15
:10F694002E2E2E2E2E2E2E2E2E2020200D0A002031
:10F6A4005241303D2E2E2E5241313D416E616C6FE0
:10F6B40067202C5241343D6C65642C5241332E2E0C
:10F6C4002E5243363D545820554152543120524312
:10F6D400373D525820554152540D0A0020412069AB
:10F6E4006E636C7572653A200D0A204469616C6F13
:10F6F4006775655F4F70657261746575725F5043BD
:10F704005F7669615F554152545F323032332D3038
:10F714003930350D0A0D0A00204469726563746F2F
:10F724007279203A433A5C4D504C4142585F5072D2
:10F734006F6A656374735C31384632374B34325FB9
:10F74400504D575F434350313233345F323032359A
:10F754000D0A0020424153452031384632374B349C
:10F7640032202B204C4344345832302B2050574DF8
:10F77400312C322C332C3420416E616C6F67205253
:10F7840041302C312C322C330D0A00204C434420C0
:10F79400347832302062757320493243312048571F
:10F7A400203A205243333D53434C2C5243343D536F
:10F7B40044410D0A002050726F6A656374203A2038
:10F7C40031384632374B34325F504D575F434350E4
:10F7D400313233345F323032350D0A0020536F75C5
:10F7E400726365203A20206D61696E2E63202C209F
:10F7F400726576203A5F3235303431330D0A002099
:10F80400436F6E6669672020496E7465726E616C21
:10F8140020466F73632036344D487A0D0A00202049
:10F8240020202020202020202020202020202020D4
:10F834002020002052423020414C45525420696E11
:10F844007075740D0A002052617070656C203A2046
:10F8540063646520504D57793D5858585820617657
:10F86400656320793D63686F697820504D57203176
:10F87400206F7520322065742020787878782020D5
:10F8840076616C657572206475747920303030301F
:10F89400206120313031350D0A0020546573742005
:10F8A400646966666572656E7465732076616C65FD
:10F8B40075727320646520447574792D6379636C63
:10F8C4006520766961206C6520636C617669657278
:10F8D400207465726D696E616C20594154200D0A63
:10F8E4000020456E7472657220756E652076616CB9
:10F8F4006575722050574D793D7878787820707509
:10F904006973203C656E7465723E20617665632080
:10F91400793D31206F75203220617520636C6176EA
:10F924006965720D0A0020496E697420494E41329E
:10F934003236206D657375726520646520636F755A
:10F9440072616E7420766961204932432C20736899
:10F95400756E74206465203135306D5620706F7576
:10F96400203135416D70730D0A002043616C69626A
:10F97400726174696F6E2072656769737465722051
:10F984003035682028706F7572207368756E742026
:10F99400302C3031206F686D202065742038204170
:10F9A4006D707329200D0A002050574D323D585870
:10F9B4005858202020617665632058585820646583
:10F9C400203030303020613130303020706F75722B
:10F9D40020524331206465203025206131303025A8
:10F9E400200D0A002050574D313D585858582020BA
:10F9F4002061766563205858582064652030303083
:10FA04003020613130303020706F757220524332B3
:10FA1400206465203025206131303025200D0A0016
:10FA24002041637469766572206C6120736F72740F
:10FA340069652050574D792061766563204D413DBD
:10FA4400312020202028617272657420766961203B
:10FA54004D413D30290D0A0020416C657274204DE2
:10FA640041534B5F454E5F5245472072656769734A
:10FA740074657220303768203C2D203234303020B9
:10FA8400706F757220302E3620410D0A0020766585
:10FA94007273696F6E2050726F746F747970652021
:10FAA4003A204C434420426C65752061206C2761E8
:10FAB400647265737365203078323720210D0A0033
:10FAC40020496E697469616C69736174696F6E2031
:10FAD40050574D312C322061766563204652657152
:10FAE40020332C394B487A202854696D65723229A9
:10FAF4000D0A00204D61736B2F416C6572742020D8
:10FB04004D41534B5F454E5F5245472072656769CF
:10FB14007374657220303668203C2D20307838307C
:10FB240030310D0A002045727265757220646520BB
:10FB3400536169736965202063686F697820434362
:10FB4400502025632076616C6575722050574D20D6
:10FB54002535640D0A0020436F6E666967202049CD
:10FB64004E413232365F434F4E465F5245472C304A
:10FB74007834334646202877617320307834313224
:10FB84003720290D0A00200D0A53657175656E63CF
:10FB940065206427496E6974204C434420347832CC
:10FBA400302076696120493243312050434638354C
:10FBB40037340D0A00204020646563696D616C2050
:10FBC400232534752020736F697420404465766959
:10FBD4006365203762697473203D203058253032C4
:10FBE400582000204368617267656D656E742063F8
:10FBF40061726163746572657320537065636961D2
:10FC040075782020656E20434752414D0D0A00202F
:10FC1400436F6D70696C65642025732061742025C1
:10FC24007320555443202076657273696F6E205893
:10FC34004338203A2564200D0A000D0A20416C61E6
:10FC4400726D204F7665725F63757272656E742093
:10FC54002E2E666169726520756E207265736574F7
:10FC64000D0A00204D413D31206F752030202020A9
:10FC7400313D4D6172636865206F7520303D41727E
:10FC84007265742050574D200D0A0020546573741A
:10FC94002070726573656E6365206465766963655B
:10FCA40073207375722042757320493243310D0AF3
:10FCB400002046696E20646520706172616D657410
:10FCC4007261676520494E413232362E2E2E204F06
:10FCD4004B0D0A0D0A002061647265737365204C34
:10FCE40043443D20256420736F69742030582530C7
:10FCF4003258200D0A0020536575696C2064276111
:10FD04006C657274652025332E336620416D7065F1
:10FD14007265730D0A00204D657375726520646504
:10FD240020636F7572616E742025203564206D41E7
:10FD3400200D0A00202A2050574D3220737572205E
:10FD44005243312028544D5232293D3025200D0A8A
:10FD540000202A2050574D312073757220524332AF
:10FD64002028544D5232293D3025200D0A00456586
:10FD740070726F6D2032344C437878782032353687
:10FD84006B206F75203531324B0020494E41204D98
:10FD9400616E7566616374756572202030782530F4
:10FDA40034580D0A0020494E41204964656E746937
:10FDB4006669616E74203078253034580D0A00204D
:10FDC4005043463837353420666F72204C43442004
:10FDD4003278313663617273000D0A2052415A2021
:10FDE400616C61726D65202C526573746172740D5F
:10FDF4000A002025332E3366205720205365756969
:10FE04006C3D25332E336620200020496E69745FD3
:10FE14004932432829203130304B687A3B0D0A009F
:10FE240050574D322D524331202025346420253340
:10FE34002E316625630050574D312D524332202018
:10FE44002534642025332E3166256300494E413222
:10FE540032362043757272656E742073656E736FEB
:10FE640072004361726163746572657320537065D7
:10FE7400636961757820002025322E326620562071
:10FE84002025322E3366204120202E00504D57323B
:10FE94002D524331202534642025332E31662563C9
:10FEA4000050574D312D52433220253464202533E0
:10FEB4002E3166256300205072657320456E74658B
:10FEC40072206B657920210D0A0056657273696F83
:10FED4006E2050726F746F747970652021005043E6
:10FEE40046383537344120386269747320492F4FBE
:10FEF400004E623D253564202050574D313D20256C
:10FF040020346400202020202020202050574D320F
:10FF14003D20252034640020495442322044697332
:10FF240061626C6564200D0A002050726573656E11
:10FF3400746174696F6E203A0D0A004C4344203298
:10FF4400313139203278313663617273002049547B
:10FF5400423220456E61626C6564200D0A00504394
:10FF6400463835373420386269747320494F004568
:10FF74004550524F4D2035313262797465730020FB
:10FF84004572726575722063780D0A004F4C4544C2
:10FF9400205353443133303600205361697369650B
:10FFA400204F4B20006E6F6E20636F6E6E752021A4
:10FFB40000417072203133203230323500525443C4
:10FFC400204453333233310031363A32373A323502
:10FFD4000048656C700D0A0052656375203A00494B
:10FFE4004E46004E414E00696E66006E616E006CB6
:0BFFF4006C7300202E31006C660000D2
:020000040001F9
:10000000D6ECB9F0000E0101A26F000E0001FA6FEC
:10001000000EF96F000EF925D96E030EFA21DA6E83
:10002000000EDF6EF94BFA2BFA5109E1800EF95DF3
:10003000D8A01DEF80F01FEF80F00AEF80F0000ED7
:10004000FA6F000EF96F800EF925D96E030EFA21B2
:10005000DA6E000EDF6EF94BFA2BFA5109E1800ED1
:10006000F95DD8A036EF80F038EF80F023EF80F014
:10007000000EFA6F000EF96F200EF925D96E020EF0
:10008000FA21DA6E000EDF6EF94BFA2BFA5109E114
:100090007F0EF95DD8A04FEF80F051EF80F03CEF7C
:1000A00080F0000EFA6F000EF96FAC0EF925D96ED4
:1000B000010EFA21DA6E000EDF6EF94BFA2BFA51BF
:1000C00009E1090EF95DD8A068EF80F06AEF80F0D1
:1000D00055EF80F0000EF76F030EF86FB9ECB7F034
:1000E00055ECAEF0000E0001FA6F000EF96FBA8801
:1000F000110E0101E86F3C0EE76FCB0EE82EFED724
:10010000E72FFCD7E82FFAD7BA98110E0101E86F54
:100110003C0EE76FCB0EE82EFED7E72FFCD7E82F7B
:10012000FAD70001F94BFA2BFA5109E1080EF95DF3
:10013000D8A09DEF80F09FEF80F077EF80F0BA8835
:10014000C7ECB6F0090E0101E86F1E0EE76FE40E72
:10015000E82EFED7E72FFCD7E82FFAD700F04EECB9
:10016000B9F04EECB9F02D0E086EFF0E096ED0EC12
:10017000B5F0000E0001FA6F000EF96FD890F93556
:10018000D96EFA35DA6EB60ED926010EDA226F0074
:1001900078FF08F06F0074FF09F0D0ECB5F00001B3
:1001A000F94BFA2BFA5109E1090EF95DD8A0DBEF02
:1001B00080F0DDEF80F0BEEF80F04EECB9F0F7C0DC
:1001C000D8F0F8C0D9F0130E0001DA6FFC0EDB6F27
:1001D000B50EDC6FFF0EDD6FCC0EDE6FFF0EDF6F36
:1001E000090EE16F380EE06FFBECB5F0F7C008F0D8
:1001F000F8C009F017ECB4F04EECB9F0020EF9ECCF
:10020000B7F0910E086EFA0E096ED0ECB5F00E0E36
:10021000086EFE0E096ED0ECB5F05FECBAF08F0EF2
:10022000086EFC0E096ED0ECB5F090EC9EF04EEC32
:10023000B9F0270E0001FC6F000E586E140E576EB9
:10024000200ED86F020ED96FDA0EDA6FFC0EDB6F5C
:10025000FCC0DCF0DD6BFCC0DEF0DF6BFBECB5F06E
:10026000200E086E020E096E17ECB4F03D01758980
:100270008A0E086EFB0E096ED0ECB5F03D01738F4F
:1002800063ECA8F04EECB9F0010E50ECB0F0010EAA
:100290002F6ECE0E306EFE0E316E010EF2ECBAF005
:1002A000020EF9ECB7F0010E50ECB0F0020E50EC7B
:1002B000B0F0090E0101E86F1E0EE76FE40EE82EA4
:1002C000FED7E72FFCD7E82FFAD700F0E70E086E2D
:1002D000FB0E096ED0ECB5F0660E286EFE0E296E90
:1002E0007BECB1F0000E2B6E000E2A6EC4ECA7F072
:1002F000000E0001FA6F000EF96F000E2B6E020E59
:100300002A6E010EF9252C6E000EFA212D6EF9C011
:100310002EF0F9ECABF00001F94BFA2BFA5109E1A0
:10032000080EF95DD8A097EF81F099EF81F07DEF8D
:1003300081F0010EF9ECB7F0C40E086EFA0E096EEA
:10034000D0ECB5F023ECBBF017ECBBF04EECB9F001
:10035000BEECB2F0D28ED28E550E086EFD0E096E36
:10036000D0ECB5F0380E086EFD0E096ED0ECB5F08D
:10037000010E50ECB0F0020E50ECB0F0000E000197
:10038000FE6F010EFD6F86C108F087C109F00A6A91
:100390000B6A000E3AECA3F008C02FF009C030F051
:1003A0000AC031F00BC032F0330E336E330E346EB0
:1003B000230E356E410E366E47EC98F02FC062F179
:1003C00030C063F131C064F132C065F186C108F01C
:1003D00087C109F0D6ECB8F0200E0001D86F020EEC
:1003E000D96F3A0EDA6FFE0EDB6F86C1DCF087C183
:1003F000DDF062C1DEF063C1DFF064C1E0F065C131
:10040000E1F0000EE36F250EE26FFBECB5F0010E9C
:100410002F6E200E306E020E316E010EE5ECBAF03A
:10042000000E0001FE6F020EFD6F84C108F085C151
:1004300009F00A6A0B6A000E3AECA3F008C02FF02C
:1004400009C030F00AC031F00BC032F0330E336E09
:10045000330E346E230E356E410E366E47EC98F037
:100460002FC05EF130C05FF131C060F132C061F188
:1004700084C108F085C109F0D6ECB8F0200E000167
:10048000D86F020ED96F240EDA6FFE0EDB6F84C1B7
:10049000DCF085C1DDF05EC1DEF05FC1DFF060C180
:1004A000E0F061C1E1F0000EE36F250EE26FFBECBE
:1004B000B5F0010E2F6E200E306E020E316E020E60
:1004C000E5ECBAF0030EF9ECB7F0010E50ECB0F029
:1004D000020E50ECB0F02A0E086EF90E096ED0EC48
:1004E000B5F014EC9AF0000E0301006F000E00014D
:1004F000F76F030EF86F010E3A01666F3901A09F86
:10050000010E3A01866F000E676F010E656F3901AB
:10051000909F000E0101716F000E706F000E9F6FB3
:100520009E0E086EF80E096ED0ECB5F0240E086E23
:10053000FA0E096ED0ECB5F0E50E086EF80E096EF5
:10054000D0ECB5F0000E0301006F000E0001F76F54
:10055000030EF86FBEECB2F07A0E0101E86FC10E27
:10056000E76F810EE82EFED7E72FFCD7E82FFAD7EA
:1005700000D00101A705D8A4C0EF82F0C2EF82F03D
:100580006EEF86F0DC0E086EFF0E096ED0ECB5F053
:10059000800E086E030E096E17ECB4F04EECB9F045
:1005A000800E0001F56F030EF66F6000D7F3D9FFE0
:1005B0006000DBF3DAFF480EDE18D8A4E2EF82F029
:1005C000E4EF82F02EEF83F020EE01F0F551D92612
:1005D000F651DA22650EDE18D8A4F1EF82F0F3EFBF
:1005E00082F02EEF83F020EE02F0F551D926F6517D
:1005F000DA226C0EDE18D8A400EF83F002EF83F04D
:100600002EEF83F020EE03F0F551D926F651DA22D1
:10061000700EDE18D8A40FEF83F011EF83F02EEFE9
:1006200083F0D50E086EFF0E096ED0ECB5F0670EA4
:10063000086EFC0E096ED0ECB5F0E80E086EF90EEF
:10064000096ED0ECB5F0AC0E086EF90E096ED0EC68
:10065000B5F0000E0001F56F000EF66F6000D7F3E5
:10066000D9FF6000DBF3DAFF520EDE18D8A43BEFAF
:1006700083F03DEF83F07AEF83F020EE01F0F55147
:10068000D926F651DA22650EDE18D8A44AEF83F097
:100690004CEF83F07AEF83F020EE05F0F551D92688
:1006A000F651DA22720EDE18D8A459EF83F05BEF10
:1006B00083F07AEF83F020EE06F0F551D926F6515B
:1006C000DA22740EDE18D8A468EF83F06AEF83F0A4
:1006D0007AEF83F0000E01019F6FBA86DD0E086E7F
:1006E000FD0E096ED0ECB5F0BA88000E0001F56F72
:1006F000000EF66F6000D7F3D9FF6000DBF3DAFF7E
:10070000500EDE18D8A487EF83F089EF83F016EF40
:1007100086F020EE01F0F551D926F651DA22570E77
:10072000DE18D8A496EF83F098EF83F016EF86F0EA
:1007300020EE02F0F551D926F651DA224D0EDE18E0
:10074000D8A4A5EF83F0A7EF83F016EF86F020EE94
:1007500004F0F551D926F651DA223D0EDE18D8A460
:10076000B4EF83F0B6EF83F016EF86F020EE03F0DF
:10077000F551D926F651DA22DF50FB6F000E010148
:10078000936F000E926FD00EE76FFF0EE86F0001BF
:10079000FB510101E96FEA6BE751E927E851EA23D0
:1007A000EA5107E10A0EE95DD8B0D9EF83F0DBEF3B
:1007B00083F011EF86F0300E0001FB65E2EF83F06D
:1007C000E4EF83F011EF86F0330EFB61EAEF83F084
:1007D000ECEF83F011EF86F00101924B932BD00EDA
:1007E000E76FFF0EE86F000120EE05F0F551D92606
:1007F000F651DA22DF500101E96FEA6BE751E92790
:10080000E851EA23EA5107E10A0EE95DD8B00BEF9F
:1008100084F00DEF84F02AEF84F0000120EE05F063
:10082000F551D926F651DA22DF500101E76FD00EDB
:10083000E725086E096AFF0E0922030E0B6EE80E0B
:100840000A6EEBECB9F008C0FDF009C0FEF0010142
:10085000924B932BD00EE76FFF0EE86F000120EE56
:1008600006F0F551D926F651DA22DF500101E96F81
:10087000EA6BE751E927E851EA23EA5107E10A0E5A
:10088000E95DD8B046EF84F048EF84F06EEF84F075
:10089000000120EE06F0F551D926F651DA22DF509C
:1008A0000101E76FE751640D6F00CCFFE8F16F00C5
:1008B000D0FFE9F10001FD510101E8270001FE51DF
:1008C0000101E923400EE8250001FD6FED0E010155
:1008D000E9210001FE6F0101924B932BD00EE76FCF
:1008E000FF0EE86F000120EE07F0F551D926F65112
:1008F000DA22DF500101E96FEA6BE751E927E8519D
:10090000EA23EA5107E10A0EE95DD8B08AEF84F0E4
:100910008CEF84F0B2EF84F0000120EE07F0F55187
:10092000D926F651DA22DF500101E76FE7510A0DAF
:100930006F00CCFFE8F16F00D0FFE9F10001FD513D
:100940000101E8270001FE510101E923200EE825FD
:100950000001FD6FFE0E0101E9210001FE6F0101A2
:10096000924B932BD00EE76FFF0EE86F000120EE45
:1009700008F0F551D926F651DA22DF500101E96F6E
:10098000EA6BE751E927E851EA23EA5107E10A0E49
:10099000E95DD8B0CEEF84F0D0EF84F0F0EF84F0D2
:1009A000000120EE08F0F551D926F651DA22DF5089
:1009B0000101E76FE7510001FD250101E86F000E1D
:1009C0000001FE210101E96FD00EE8250001FD6F55
:1009D000FF0E0101E9210001FE6F0101924B932BF3
:1009E000050E92199311D8A4F8EF84F0FAEF84F071
:1009F000F3EF85F0F80E0001FD5D030EFE59D8B04F
:100A000004EF85F006EF85F0F3EF85F0BC8AC0EFC8
:100A100085F09D0E086EFF0E096ED0ECB5F0FDC09E
:100A200086F1FEC087F1FDC008F0FEC009F00A6A39
:100A30000B6A000E3AECA3F008C02FF009C030F0AA
:100A40000AC031F00BC032F0330E336E330E346E09
:100A5000230E356E410E366E47EC98F02FC062F1D2
:100A600030C063F131C064F132C065F1200E000185
:100A7000D86F020ED96FA50EDA6FFE0EDB6F86C13E
:100A8000DCF087C1DDF062C1DEF063C1DFF064C17C
:100A9000E0F065C1E1F0000EE36F250EE26FFBECC4
:100AA000B5F0010E2F6E200E306E020E316E010E6B
:100AB000E5ECBAF086C108F087C109F0D6ECB8F0D1
:100AC000D6EF85F0FDC084F1FEC085F1FDC008F0D1
:100AD000FEC009F00A6A0B6A000E3AECA3F008C0E7
:100AE0002FF009C030F00AC031F00BC032F0330EE5
:100AF000336E330E346E230E356E410E366E47EC78
:100B000098F02FC05EF130C05FF131C060F132C0AB
:100B100061F1200E0001D86F020ED96F900EDA6FCE
:100B2000FE0EDB6F84C1DCF085C1DDF05EC1DEF05E
:100B30005FC1DFF060C1E0F061C1E1F0000EE36F82
:100B4000250EE26FFBECB5F0010E2F6E200E306E1D
:100B5000020E316E020EE5ECBAF084C108F085C1D8
:100B600009F0BEECB8F0D6EF85F0000E0001FB6F87
:100B7000830E086EFF0E096ED0ECB5F0D6EF85F04F
:100B8000FB510101E76FE86BE851000AD8B4CBEFE5
:100B900085F0B5EF85F0E751310AD8B409EF85F05B
:100BA000030AD8B462EF85F0B5EF85F00001FB5180
:100BB000D8B4DDEF85F0DFEF85F0F0EF85F0200EA3
:100BC000086E020E096E17ECB4F04EECB9F0D00EC0
:100BD0000101E76FC90EE82EFED7E72FFCD700D042
:100BE000BC9A11EF86F0200E0001D86F020ED96F6B
:100BF000290EDA6FFB0EDB6FFBC0DCF0DD6BFDC096
:100C0000DEF0FEC0DFF0FBECB5F0200E086E020E49
:100C1000096E17ECB4F04A0E086EF80E096ED0ECAF
:100C2000B5F0000E0001F56F000EF66F6000D7F30F
:100C3000D9FF6000DBF3DAFF4D0EDE18D8A423EFF6
:100C400086F025EF86F069EF86F020EE01F0F55191
:100C5000D926F651DA22410EDE18D8A432EF86F0FA
:100C600034EF86F069EF86F020EE02F0F551D926D8
:100C7000F651DA223D0EDE18D8A441EF86F043EF9C
:100C800086F069EF86F020EE03F0F551D926F65193
:100C9000DA22DF50FB6F310EFB19D8A452EF86F039
:100CA00054EF86F05DEF86F0BA86510E086EFF0EA7
:100CB000096ED0ECB5F064EF86F01B0E086EFF0EE7
:100CC000096ED0ECB5F0BA96000E0001F56F000E7B
:100CD000F66F000E0101A76FC1EF87F0000E020151
:100CE000206F200E0001D86F020ED96FF50EDA6F5B
:100CF000FE0EDB6F8EC1DCF08FC1DDF086C1DEF051
:100D000087C1DFF0FBECB5F0010E2F6E200E306EC8
:100D1000020E316E010EE5ECBAF0200E086E020EE6
:100D2000096E17ECB4F0200E0001D86F020ED96FD7
:100D3000080EDA6FFF0EDB6F84C1DCF085C1DDF0D9
:100D4000FBECB5F0010E2F6E200E306E020E316EF0
:100D5000020EE5ECBAF0200E086E020E096E17ECDA
:100D6000B4F0E0EC9FF0270E0001FC6F000E1A6E4D
:100D7000000E1B6EA00E1C6E3F0E1D6E74C108F09F
:100D800075C109F00A6A0B6A000E3AECA3F008C0BC
:100D900016F009C017F00AC018F00BC019F020ECCB
:100DA00096F016C02FF017C030F018C031F019C0FF
:100DB00032F0000E336E000E346E7A0E356E440E35
:100DC000366E47EC98F02FC03EF130C03FF131C095
:100DD00040F132C041F1000E1A6E000E1B6E200E63
:100DE0001C6E400E1D6E76C108F077C109F0000E32
:100DF00009BEFF0E0A6E0B6E010E3AECA3F008C09E
:100E000016F009C017F00AC018F00BC019F020EC5A
:100E100096F016C02FF017C030F018C031F019C08E
:100E200032F0000E336E400E346E1C0E356E460EE0
:100E3000366E47EC98F02FC042F130C043F131C01C
:100E400044F132C045F1200E0001D86F020ED96F77
:100E50007B0EDA6FFE0EDB6F3EC1DCF03FC1DDF0D2
:100E600040C1DEF041C1DFF042C1E0F043C1E1F03A
:100E700044C1E2F045C1E3F0FBECB5F001019F0590
:100E8000D8A445EF87F047EF87F066EF87F04F0E65
:100E90000201336FBA96000E0101876F000E866F54
:100EA000000E856F000E846F000E096E000E086E36
:100EB000D6ECB8F0000E096E000E086EBEECB8F06D
:100EC0003E0E086EFC0E096ED0ECB5F0200E086EDA
:100ED000020E096E17ECB4F0010E2F6E200E306E6C
:100EE000020E316E030EE5ECBAF03EC116F03FC1C2
:100EF00017F040C118F041C119F042C11AF043C1C6
:100F00001BF044C11CF045C11DF020EC96F016C04A
:100F100046F117C047F118C048F119C049F1200E39
:100F20000001D86F020ED96FF60EDA6FFD0EDB6F7F
:100F300046C1DCF047C1DDF048C1DEF049C1DFF059
:100F40003AC1E0F03BC1E1F03CC1E2F03DC1E3F069
:100F5000FBECB5F0200E086E020E096E17ECB4F033
:100F6000010E2F6E200E306E020E316E040EE5EC77
:100F7000BAF0000E0201206F4EECB9F001018E4B69
:100F80008F2BBC8A090E0101E86F1E0EE76FE40E7D
:100F9000E82EFED7E72FFCD7E82FFAD700F0BC9A4F
:100FA000A2EF82F057EF00F0000E00018B6F000EF1
:100FB0008A6F6CC09CF06DC09DF06EC09EF06FC0DB
:100FC0009FF09FBFE8EF87F0E6EF87F0FEEF87F036
:100FD000000E8B6F010E8A6F9CC008F09DC009F057
:100FE0009EC00AF09FC00BF06DECB8F008C09CF0FA
:100FF00009C09DF00AC09EF00BC09FF0000E0001DA
:10100000A36F000EA26F6CC18EF06DC18FF08A517C
:101010008B11D8A40EEF88F010EF88F017EF88F04E
:1010200054A415EF88F017EF88F031EF88F08A515B
:101030008B11D8A41EEF88F020EF88F026EF88F0FF
:10104000000E776F2B0E766F2AEF88F0000E776F09
:101050002D0E766F76C0A0F2A24BA32B8E07D8A0E0
:101060008F079CC008F09DC009F09EC00AF09FC089
:101070000BF096ECAAF008040910D8A442EF88F00F
:1010800044EF88F08EEF88F0BF0E0001716FFF0E05
:10109000726F7051736F746B715173277251742337
:1010A000745107E11A0E735DD8B059EF88F05BEF09
:1010B00088F069EF88F0A00EA2250C6E020EA32125
:1010C0000D6EE30E0E6EFF0E0F6E86ECB4F075EF34
:1010D00088F0A00EA2250C6E020EA3210D6EEB0E61
:1010E0000E6EFF0E0F6E86ECB4F00001FD0E8E2723
:1010F000FF0E8F236AC018F06BC019F0A00E1A6E95
:10110000020E1B6E8EC01CF08FC01DF099ECADF06E
:1011100018C06AF019C06BF0DBEF8DF09CC008F0CE
:101120009DC009F09EC00AF09FC00BF096ECAAF09B
:1011300008500910D8A49FEF88F0A1EF88F0D4EFF1
:1011400088F0BF0E0001716FFF0E726F7051736FE8
:10115000746B7151732772517423745107E11A0E25
:10116000735DD8B0B6EF88F0B8EF88F0C6EF88F0BE
:10117000A00EA2250C6E020EA3210D6EE70E0E6EC0
:10118000FF0E0F6E86ECB4F075EF88F0A00EA2256E
:101190000C6E020EA3210D6EEF0E0E6EFF0E0F6E83
:1011A00086ECB4F075EF88F0000E0001A46F000E1D
:1011B000A56F800EA66F3F0EA76F000EA16F000EE9
:1011C000A06F9CC008F09DC009F09EC00AF09FC0AF
:1011D0000BF0000E0C6E000E0D6E000E0E6E000E6B
:1011E0000F6E08ECAFF0D8B0F8EF88F0FAEF88F0A7
:1011F0007DEF89F019EF89F0A4C016F0A5C017F0B3
:10120000A6C018F0A7C019F0000E1A6E000E1B6ED3
:10121000200E1C6E410E1D6E20EC96F016C0A4F040
:1012200017C0A5F018C0A6F019C0A7F00001A04B88
:10123000A12B9CC02FF09DC030F09EC031F09FC00C
:1012400032F0000E1A6E000E1B6E200E1C6E410E48
:101250001D6EA4C016F0A5C017F0A6C018F0A7C058
:1012600019F020EC96F016C033F017C034F018C017
:1012700035F019C036F014ECAAF0D8B042EF89F07E
:1012800044EF89F0FCEF88F064EF89F0A4C02FF000
:10129000A5C030F0A6C031F0A7C032F0000E336E0A
:1012A000000E346E200E356E410E366E47EC98F00F
:1012B0002FC0A4F030C0A5F031C0A6F032C0A7F016
:1012C0000001A007D8A0A1079CC02FF09DC030F05E
:1012D0009EC031F09FC032F0A4C033F0A5C034F0FE
:1012E000A6C035F0A7C036F014ECAAF0D8A07BEF6A
:1012F00089F07DEF89F046EF89F070C00EF00F6A3B
:101300000EECB7F00E500001916F91C090F0670E97
:101310009119D8A48EEF89F090EF89F0B6EF89F09B
:1013200052505310D8A497EF89F099EF89F09DEFB0
:1013300089F0000E536E010E526E53BEAAEF89F073
:10134000535006E15204D8B0A8EF89F0AAEF89F013
:10135000B0EF89F0000E8D6F060E8C6FBFEF89F035
:1013600052C08CF053C08DF0BFEF89F053BEBBEF7D
:1013700089F0BDEF89F0AAEF89F0B0EF89F0670E30
:101380009119D8A4C6EF89F0C8EF89F0F7EF89F07A
:10139000A1AFD6EF89F0FC0EA05DFF0EA159D8A039
:1013A000D4EF89F0D6EF89F0F5EF89F0FF0E716F79
:1013B000FF0E726F8CC073F08DC074F07151732783
:1013C00072517423A051735D7451800A756FA151DD
:1013D000800A7559D8A0EFEF89F0F1EF89F0F5EFA9
:1013E00089F0660E906FF7EF89F0650E906F8CC0F4
:1013F00082F08DC083F0670E9119D8A402EF8AF0B5
:1014000004EF8AF014EF8AF0660E9019D8A40BEF5F
:101410008AF00DEF8AF016EF8AF0A1BF14EF8AF080
:1014200012EF8AF016EF8AF0824B832B660E90192A
:10143000D8A41DEF8AF01FEF8AF03FEF8AF0A1BF1A
:1014400026EF8AF024EF8AF032EF8AF0000EA46FC4
:10145000000EA56F800EA66F3F0EA76F000EA16F46
:10146000000EA06F670E9119D8B439EF8AF03BEFE8
:101470008AF03FEF8AF0A0518227A1518323000E0A
:101480009B6F000E9A6F9CC092F09DC093F09EC01F
:1014900094F09FC095F0A4C084F0A5C085F0A6C0CC
:1014A00086F0A7C087F0D0EF8AF092C02FF093C0EB
:1014B00030F094C031F095C032F0A4C033F0A5C034
:1014C00034F0A6C035F0A7C036F047EC98F02FC036
:1014D00048F030C049F031C04AF032C04BF02FEC38
:1014E000A1F048C096F049C097F04AC098F04BC0B0
:1014F00099F096C008F097C009F098C00AF099C01A
:101500000BF091ECA9F008C088F009C089F092C0F6
:101510002FF093C030F094C031F095C032F0A4C0E9
:101520001AF0A5C01BF0A6C01CF0A7C01DF096C005
:1015300016F097C017F098C018F099C019F020EC79
:1015400096F016C033F017C034F018C035F019C04B
:1015500036F031ECB7F02FC092F030C093F031C0CC
:1015600094F032C095F0A4C02FF0A5C030F0A6C012
:1015700031F0A7C032F0000E336E000E346E200E34
:10158000356E410E366E47EC98F02FC0A4F030C097
:10159000A5F031C0A6F032C0A7F000019A4B9B2BFA
:1015A00082519A5D9B51800A716F8351800A7159F3
:1015B000D8A0DDEF8AF0DFEF8AF055EF8AF0A4C003
:1015C00016F0A5C017F0A6C018F0A7C019F0000EBD
:1015D0001A6E000E1B6EA00E1C6E400E1D6E20ECCF
:1015E00096F016C096F017C097F018C098F019C082
:1015F00099F092C02FF093C030F094C031F095C0B4
:1016000032F096C033F097C034F098C035F099C0EE
:1016100036F014ECAAF0D8B010EF8BF012EF8BF08C
:101620001DEF8BF0000E0001966F000E976F000EFD
:10163000986F000E996F46EF8BF092C008F093C040
:1016400009F094C00AF095C00BF096C00CF097C05A
:101650000DF098C00EF099C00FF008ECAFF0D8A0D4
:1016600034EF8BF036EF8BF046EF8BF0000188B152
:101670003CEF8BF03EEF8BF046EF8BF0000E966F59
:10168000000E976F000E986F000E996F9CC008F0C7
:101690009DC009F09EC00AF09FC00BF096C00CF0F0
:1016A00097C00DF098C00EF099C00FF0C0EC93F009
:1016B00008C092F009C093F00AC094F00BC095F0F6
:1016C00092C02FF093C030F094C031F095C032F04A
:1016D000000E1A6E000E1B6E200E1C6E410E1D6E4B
:1016E00084C016F085C017F086C018F087C019F0C6
:1016F00020EC96F016C033F017C034F018C035F067
:1017000019C036F014ECAAF0D8A089EF8BF08BEF5B
:101710008BF0B4EF8BF00001A04BA12B84C016F02E
:1017200085C017F086C018F087C019F0000E1A6E39
:10173000000E1B6E200E1C6E410E1D6E20EC96F0EE
:1017400016C084F017C085F018C086F019C087F065
:10175000660E00019019D8A4B0EF8BF0B2EF8BF0B9
:10176000B4EF8BF0824B832B84C0A4F085C0A5F02E
:1017700086C0A6F087C0A7F0650E00019019D8B406
:10178000C4EF8BF0C6EF8BF0CCEF8BF0A0C080F0F5
:10179000A1C081F0D0EF8BF0000E816F000E806F42
:1017A000000E7F6F000E7E6F000E7D6F000E7C6F4F
:1017B000000E9B6F000E9A6FCCEF8CF092C02FF052
:1017C00093C030F094C031F095C032F0A4C033F033
:1017D000A5C034F0A6C035F0A7C036F047EC98F0AD
:1017E0002FC048F030C049F031C04AF032C04BF051
:1017F0002FECA1F048C096F049C097F04AC098F08D
:101800004BC099F096C008F097C009F098C00AF054
:1018100099C00BF091ECA9F008C088F009C089F0DC
:1018200054B815EF8CF017EF8CF035EF8CF0000109
:1018300088518911D8A41FEF8CF021EF8CF035EF7F
:101840008CF0670E9119D8A428EF8CF02AEF8CF059
:1018500035EF8CF081BF31EF8CF02FEF8CF035EF4E
:101860008CF07C4B7D2B80EF8CF000017E517F1142
:10187000D8A43DEF8CF03FEF8CF069EF8CF081BF86
:1018800046EF8CF044EF8CF069EF8CF0A00EA225AF
:10189000D96E020EA321DA6E2E0EDF6EA24BA32BA1
:1018A0008E07D8A08F07000E7F6F010E7E6F69EF45
:1018B0008CF0A00EA225D96E020EA321DA6E300E96
:1018C000DF6EA24BA32B8E07D8A08F077C07D8A072
:1018D0007D077C517D11D8A470EF8CF072EF8CF0F5
:1018E00059EF8CF0A00EA225D96E020EA321DA6E5C
:1018F0008851300FDF6EA24BA32B8E07D8A08F0725
:1019000092C02FF093C030F094C031F095C032F007
:10191000A4C01AF0A5C01BF0A6C01CF0A7C01DF003
:1019200096C016F097C017F098C018F099C019F03B
:1019300020EC96F016C033F017C034F018C035F024
:1019400019C036F031ECB7F02FC092F030C093F0F0
:1019500031C094F032C095F0A4C02FF0A5C030F093
:10196000A6C031F0A7C032F0000E336E000E346E08
:10197000200E356E410E366E47EC98F02FC0A4F065
:1019800030C0A5F031C0A6F032C0A7F0000180073A
:10199000D8A081079A4B9B2B82519A5D9B51800A5C
:1019A000716F8351800A7159D8B0D9EF8CF0DBEF99
:1019B0008CF0E9EF8CF0A3BFE7EF8CF0A35109E1C5
:1019C0004B0EA25DD8A0E7EF8CF0E9EF8CF0DEEFD4
:1019D0008BF07E517F11D8A4F0EF8CF0F2EF8CF0F9
:1019E00003EF8DF054A8F7EF8CF0F9EF8CF003EFD4
:1019F0008DF0A00EA225D96E020EA321DA6E2E0E56
:101A0000DF6EA24BA32BA00EA225D96E020EA3213E
:101A1000DA6E000EDF6E650E9019D8A412EF8DF00D
:101A200014EF8DF07AEF88F0000E9B6F4F0E9A6FD7
:101A3000A00E9A25D96E020E9B21DA6E000EDF6E83
:101A4000000E8B6F000E8A6FA1BF2BEF8DF029EF78
:101A50008DF033EF8DF0000E8B6F010E8A6FA06D4D
:101A6000A11FD8B0A12B000E8D6F020E8C6F64EFFA
:101A70008DF09A07D8A09B07A00E9A25D96E020E6A
:101A80009B21DA6EA0C008F0A1C009F0000E0B6E19
:101A90000A0E0A6EB0ECAEF00850300FDF6EA0C038
:101AA00008F0A1C009F0000E0B6E0A0E0A6E37ECAA
:101AB000ADF008C0A0F009C0A1F000018C07D8A0CB
:101AC0008D078E07D8A08F07A051A111D8A46BEF66
:101AD0008DF06DEF8DF039EF8DF08DBF7AEF8DF0D9
:101AE0008D5106E18C05D8B078EF8DF07AEF8DF04E
:101AF00039EF8DF09A07D8A09B078A518B11D8A493
:101B000084EF8DF086EF8DF08CEF8DF0000E796F05
:101B10002B0E786F90EF8DF0000E796F2D0E786F91
:101B2000A00E9A25D96E020E9B21DA6E6000E3F1B9
:101B3000DFFF8E07D8A08F079A07D8A09B07BF0E9C
:101B4000716FFF0E726F7051736F746B71517327E9
:101B500072517423745109E11A0E735DD8A0B3EF6A
:101B60008DF0B5EF8DF0BBEF8DF0000E7B6F650E45
:101B70007A6FBFEF8DF0000E7B6F450E7A6FA00E6F
:101B80009A25D96E020E9B21DA6E6000EBF1DFFF21
:101B90008E07D8A08F07A00EA2250C6E020EA321DF
:101BA0000D6EA00E9A250E6E020E9B210F6E86EC16
:101BB000B4F07AEF88F012006000ABF2D9FF600059
:101BC000AFF2DAFF6F007BFFF6FF6F0077FFF7FFE2
:101BD000000EF86E0800F550250AD8A4F2EF8DF03B
:101BE000F4EF8DF09CEF93F06000ABF2D9FF600052
:101BF000AFF2DAFFDE2A000EDD22000E01016D6F6A
:101C0000000E6C6F6CC154F06DC155F05268536892
:101C1000000E0001BD6F000EBC6F5DEF8EF05480B2
:101C20006000ABF2D9FF6000AFF2DAFFDE2A000EEF
:101C3000DD225DEF8EF0548210EF8EF0548410EFB1
:101C40008EF0548610EF8EF0548810EF8EF0000E58
:101C5000BD6F010EBC6F5DEF8EF06000ABF2D9FF7F
:101C60006000AFF2DAFF6F007BFFF6FF6F0077FFD7
:101C7000F7FF000EF86E0800F550AE6FAF6BAF5176
:101C8000000AD8B446EF8EF027EF8EF0AE51200A4E
:101C9000D8B421EF8EF0030AD8B424EF8EF0080AEE
:101CA000D8B41EEF8EF0060AD8B40FEF8EF01D0ADE
:101CB000D8B41BEF8EF027EF8EF0BC51BD11D8B415
:101CC00064EF8EF066EF8EF02DEF8EF054A06BEF88
:101CD0008EF06DEF8EF06EEF8EF054926000ABF2EE
:101CE000D9FF6000AFF2DAFF6F007BFFF6FF6F00F5
:101CF00077FFF7FF000EF86E0800F5502A0AD8A407
:101D000084EF8EF086EF8EF0BAEF8EF06000ABF2CB
:101D1000D9FF6000AFF2DAFFDE2A000EDD2260009C
:101D2000B3F2D9FF6000B7F2DAFF6F007CFFAEF0CC
:101D3000020EDE266F007CFFAFF0000EDD22600099
:101D4000BBF2D9FF6000BFF2DAFF6F0078FF6CF1E1
:101D50006F0074FF6DF101016DBFB3EF8EF0B1EF55
:101D60008EF0FDEF8EF054806C6D6D1FD8B06D2B32
:101D7000FDEF8EF06000ABF2D9FF6000AFF2DAFF4A
:101D80006F0078FF0FF06F0074FF10F0AAECA5F061
:101D90000FC06CF110C06DF1D7EF8EF06000ABF2A8
:101DA000D9FF6000AFF2DAFFDE2A000EDD22D00E8E
:101DB0000001AE6FFF0EAF6F6000ABF2D9FF6000A5
:101DC000AFF2DAFF6F007BFFF6FF6F0077FFF7FFE0
:101DD000000EF86E0800F550B06FB16BAE51B02731
:101DE000AF51B123B15109E10A0EB05DD8A0FBEFAC
:101DF0008EF0FDEF8EF0CEEF8EF06000ABF2D9FFEB
:101E00006000AFF2DAFF6F007BFFF6FF6F0077FF35
:101E1000F7FF000EF86E0800F5502E0AD8A413EF55
:101E20008FF015EF8FF0A4EF8FF0000E536E000EC1
:101E3000526E6000ABF2D9FF6000AFF2DAFFDE2A2B
:101E4000000EDD226000ABF2D9FF6000AFF2DAFFD6
:101E50006F007BFFF6FF6F0077FFF7FF000EF86E55
:101E60000800F5502A0AD8A438EF8FF03AEF8FF027
:101E700061EF8FF06000ABF2D9FF6000AFF2DAFFE4
:101E8000DE2A000EDD226000B3F2D9FF6000B7F257
:101E9000DAFF6F007CFFAEF0020EDE266F007CFFE3
:101EA000AFF0000EDD226000BBF2D9FF6000BFF290
:101EB000DAFF6F0078FF52F06F0074FF53F0A4EF69
:101EC0008FF06000ABF2D9FF6000AFF2DAFF6F0075
:101ED00078FF0FF06F0074FF10F0AAECA5F00FC0B0
:101EE00052F010C053F07EEF8FF06000ABF2D9FFDC
:101EF0006000AFF2DAFFDE2A000EDD22D00E000114
:101F0000AE6FFF0EAF6F6000ABF2D9FF6000AFF2B3
:101F1000DAFF6F007BFFF6FF6F0077FFF7FF000E21
:101F2000F86E0800F550B06FB16BAE51B027AF51ED
:101F3000B123B15109E10A0EB05DD8A0A2EF8FF034
:101F4000A4EF8FF075EF8FF06000ABF2D9FF600067
:101F5000AFF2DAFF6F007BFFF6FF6F0077FFF7FF4E
:101F6000000EF86E0800F5500E6E0F6A0EECB7F01A
:101F70000E500001CC6FCC51D8B4C1EF8FF0C3EF3D
:101F80008FF00DEF90F06000ABF2D9FF6000AFF280
:101F9000DAFF6F0078FFAEF06F0074FFAFF0010E54
:101FA000AE27000EAF236000BBF2F6FF6000BFF269
:101FB000F7FF000EF86E0800F5500E6E0F6A0EEC7B
:101FC000B7F00E500001CD6FCD51D8B4EAEF8FF0CD
:101FD000ECEF8FF00DEF90F06000ABF2D9FF6000F6
:101FE000AFF2DAFF6F0078FFAEF06F0074FFAFF072
:101FF000020EAE27000EAF236000BBF2F6FF6000BA
:10200000BFF2F7FF000EF86E0800F5500E6E0F6A73
:102010000EECB7F00E500001CE6F6000ABF2D9FFAE
:102020006000AFF2DAFF6F007BFFF6FF6F0077FF13
:10203000F7FF000EF86E0800F550630AD8A423EFEE
:1020400090F025EF90F054EF90F06000ABF2D9FFE4
:102050006000AFF2DAFFDE2A000EDD226000B3F28C
:10206000D9FF6000B7F2DAFF6F007CFFAEF0020E1E
:10207000DE266F007CFFAFF0000EDD226000BBF2B9
:10208000D9FF6000BFF2DAFFDF50CF6FA8C011F0B8
:10209000A9C012F0CFC013F064ECACF011C0A8F0EE
:1020A00012C0A9F0BFEF93F06000ABF2D9FF60005F
:1020B000AFF2DAFF6F007BFFF6FF6F0077FFF7FFED
:1020C000000EF86E0800F550640AD8B46AEF90F07C
:1020D0006CEF90F084EF90F06000ABF2D9FF6000FD
:1020E000AFF2DAFF6F007BFFF6FF6F0077FFF7FFBD
:1020F000000EF86E0800F550690AD8A482EF90F03F
:1021000084EF90F0CEEF90F06000ABF2D9FF60006A
:10211000AFF2DAFFDE2A000EDD226000B3F2D9FF53
:102120006000B7F2DAFF6F007CFFAEF0020EDE2631
:102130006F007CFFAFF0000EDD226000BBF2D9FF24
:102140006000BFF2DAFF6F0078FFB2F06F0074FF3B
:10215000B3F0000EB3BFFF0EB46FB56FB66FB76FBD
:10216000B86FB96FA8C023F0A9C024F0B2C025F0A1
:10217000B3C026F0B4C027F0B5C028F0B6C029F02F
:10218000B7C02AF0B8C02BF0B9C02CF0CEEC9BF051
:1021900023C0A8F024C0A9F0BFEF93F0660ECC19BD
:1021A000D8A4D5EF90F0D7EF90F02AEF91F060002F
:1021B000ABF2D9FF6000AFF2DAFF6F007BFFF6FFF2
:1021C0006F0077FFF7FF000EF86E08006F00D4FF76
:1021D000CFF06000ABF2D9FF6000AFF2DAFFDE2A89
:1021E000000EDD226000B3F2D9FF6000B7F2DAFF23
:1021F0006F007CFFAEF0040EDE266F007CFFAFF0B8
:10220000000EDD226000BBF2D9FF6000BFF2DAFFF2
:102210006F0078FFC8F06F0078FFC9F06F0078FF9B
:10222000CAF06F0078FFCBF0A8C06AF0A9C06BF0CD
:10223000C8C06CF0C9C06DF0CAC06EF0CBC06FF002
:10224000CFC070F0D4EC87F06AC0A8F06BC0A9F0E2
:10225000BFEF93F0CC0E086E000E096EFB0E0A6EF7
:10226000FF0E0B6E000E0D6E020E0C6E1BECA7F037
:1022700008500910D8A43FEF91F041EF91F0D5EF4D
:1022800091F06000ABF2D9FF6000AFF2DAFF6F00AF
:1022900078FFAEF06F0074FFAFF0010E0001AE27C3
:1022A000000EAF236000BBF2F6FF6000BFF2F7FF45
:1022B000000EF86E08006F00D4FFCFF0BF0EAE6FB7
:1022C000FF0EAF6F6000ABF2D9FF6000AFF2DAFF34
:1022D0006F007BFFF6FF6F0077FFF7FF000EF86ED1
:1022E0000800F550B06FB16BAE51B027AF51B123BC
:1022F000B15107E11A0EB05DD8B081EF91F083EFD4
:1023000091F0A7EF91F06000B3F2D9FF6000B7F24F
:10231000DAFF6F007CFFAEF0040EDE266F007CFF5C
:10232000AFF0000EDD226000BBF2D9FF6000BFF20B
:10233000DAFF6F0078FFC8F06F0078FFC9F06F0018
:1023400078FFCAF06F0078FFCBF0C9EF91F0600022
:10235000B3F2D9FF6000B7F2DAFF6F007CFFAEF096
:10236000040EDE266F007CFFAFF0000EDD22600061
:10237000BBF2D9FF6000BFF2DAFF6F0078FFC8F050
:102380006F0078FFC9F06F0078FFCAF06F0078FF28
:10239000CBF0020E6000ABF2D9FF6000AFF2DAFFC3
:1023A000DE26000EDD2214EF91F06000ABF2D9FFC3
:1023B0006000AFF2DAFF6F007BFFF6FF6F0077FF80
:1023C000F7FF000EF86E0800F550730AD8B4EBEF73
:1023D00091F0EDEF91F00CEF92F06000ABF2D9FFCD
:1023E0006000AFF2DAFF6F0078FF08F06F0074FF53
:1023F00009F0F30E0A6EFF0E0B6E000E0D6E030E4B
:102400000C6E1BECA7F008500910D8A40AEF92F04C
:102410000CEF92F066EF92F06000ABF2D9FF600033
:10242000AFF2DAFF6F007BFFF6FF6F0077FFF7FF79
:10243000000EF86E0800F550730AD8B422EF92F03F
:1024400024EF92F02BEF92F0000E0001BF6F030E0D
:10245000BE6F30EF92F0000E0001BF6F010EBE6F35
:102460006000ABF2D9FF6000AFF2DAFFBE51DE26AA
:10247000BF51DD226000B3F2D9FF6000B7F2DAFF8E
:102480006F007CFFAEF0020EDE266F007CFFAFF027
:10249000000EDD226000BBF2D9FF6000BFF2DAFF60
:1024A0006F0078FFBAF06F0074FFBBF0A8C011F0A6
:1024B000A9C012F0BAC013F0BBC014F014ECA4F021
:1024C00011C0A8F012C0A9F0BFEF93F06000ABF20A
:1024D000D9FF6000AFF2DAFF6F007BFFF6FF6F00FD
:1024E00077FFF7FF000EF86E0800F550750AD8A4C4
:1024F0007CEF92F07EEF92F0CAEF92F06000ABF2C8
:10250000D9FF6000AFF2DAFFDE2A000EDD226000A4
:10251000B3F2D9FF6000B7F2DAFF6F007CFFAEF0D4
:10252000020EDE266F007CFFAFF0000EDD226000A1
:10253000BBF2D9FF6000BFF2DAFF6F0078FFB0F0A6
:102540006F0074FFB1F0B0C0C0F0B1C0C1F00001C5
:10255000C26BC36BC46BC56BC66BC76BA8C023F0E3
:10256000A9C024F0C0C025F0C1C026F0C2C027F029
:10257000C3C028F0C4C029F0C5C02AF0C6C02BF0E3
:10258000C7C02CF03AECA2F023C0A8F024C0A9F0F8
:10259000BFEF93F06000ABF2D9FF6000AFF2DAFF5B
:1025A0006F007BFFF6FF6F0077FFF7FF000EF86EFE
:1025B0000800F550780AD8B4E0EF92F0E2EF92F01C
:1025C000FAEF92F06000ABF2D9FF6000AFF2DAFFF1
:1025D0006F007BFFF6FF6F0077FFF7FF000EF86ECE
:1025E0000800F550580AD8A4F8EF92F0FAEF92F0EC
:1025F0005AEF93F06000ABF2D9FF6000AFF2DAFF60
:102600006F007BFFF6FF6F0077FFF7FF000EF86E9D
:1026100008006F00D4FFCFF06000ABF2D9FF60007C
:10262000AFF2DAFFDE2A000EDD226000B3F2D9FF3E
:102630006000B7F2DAFF6F007CFFAEF0020EDE261C
:102640006F007CFFAFF0000EDD226000BBF2D9FF0F
:102650006000BFF2DAFF6F0078FFB0F06F0074FF28
:10266000B1F0B0C0C0F0B1C0C1F00001C26BC36B2B
:10267000C46BC56BC66BC76BA8C023F0A9C024F0A0
:10268000C0C025F0C1C026F0C2C027F0C3C028F0EA
:10269000C4C029F0C5C02AF0C6C02BF0C7C02CF0BA
:1026A000CFC02DF03EEC9DF023C0A8F024C0A9F0CF
:1026B000BFEF93F06000ABF2D9FF6000AFF2DAFF3A
:1026C0006F007BFFF6FF6F0077FFF7FF000EF86EDD
:1026D0000800F550250AD8A470EF93F072EF93F03C
:1026E0008CEF93F06000ABF2D9FF6000AFF2DAFF3D
:1026F000DE2A000EDD22000E096E250E086EA8C02F
:102700000AF0A9C00BF08DECABF0000E0001A96F30
:10271000010EA86FBFEF93F06000ABF2D9FF60002D
:10272000AFF2DAFFDE2A000EDD22000E0001A96FF3
:10273000000EA86FBFEF93F06000ABF2D9FF60000E
:10274000AFF2DAFF6F007BFFF6FF6F0077FFF7FF56
:10275000000EF86E0800F550086E096AA8C00AF06D
:10276000A9C00BF08DECABF06000ABF2D9FF6000BC
:10277000AFF2DAFFDE2A000EDD2285EF93F01200C1
:102780000B50800B146E0B500B24166E0AAECBEF61
:1027900093F0CDEF93F0CEEF93F016801650D8B4AF
:1027A000D4EF93F0D6EF93F0EBEF93F01628D8A484
:1027B000DCEF93F0DEEF93F0E6EF93F0000E086E9F
:1027C000000E096E000E0A6E000E0B6E0A8E000ED1
:1027D0000B6EF3EF93F0000E086E000E096E000E04
:1027E0000A6E000E0B6E0F50800B156E14501518EC
:1027F000D8B4FDEF93F0FFEF93F000EF94F0148C5A
:102800000F500F24156E0EAE08EF94F00AEF94F0FF
:102810000BEF94F015801550D8B411EF94F013EF2E
:1028200094F028EF94F01528D8A419EF94F01BEF3A
:1028300094F023EF94F0000E0C6E000E0D6E000E5F
:102840000E6E000E0F6E0E8E000E0F6E30EF94F0B7
:10285000000E0C6E000E0D6E000E0E6E000E0F6E52
:102860001650155CD8B037EF94F039EF94F060EF64
:1028700094F014AC3EEF94F040EF94F042EF94F0FB
:10288000800E141A16C017F015C016F017C015F0F8
:1028900008C017F00CC008F017C00CF009C017F002
:1028A0000DC009F017C00DF00AC017F00EC00AF0F5
:1028B00017C00EF00BC017F00FC00BF017C00FF0D1
:1028C000000E176E165015C010F0116A105E000E43
:1028D000115A11BE75EF94F0115009E11A0E105CF7
:1028E000D8A075EF94F077EF94F0AEEF94F0085025
:1028F00009100A100B10D8A480EF94F083EF94F025
:10290000010E84EF94F0000E176E000E086E000E9C
:10291000096E000E0A6E000E0B6E15C016F0B7EFB2
:1029200094F017A096EF94F098EF94F09EEF94F047
:10293000D89017300109176EA0EF94F0D890173295
:1029400008A0A5EF94F0A7EF94F0A8EF94F0178EED
:102950000B340B320A3209320832162A1550165C33
:10296000D8A0B5EF94F0B7EF94F091EF94F014BCC9
:10297000BCEF94F0BEEF94F0FEEF94F01650D8A4A4
:10298000C4EF94F0C6EF94F0D0EF94F0000E086E10
:10299000000E096E000E0A6E000E0B6E1FEF96F011
:1029A0000C5008260D5009220E500A220F500B22FF
:1029B0000BA0DDEF94F0DFEF94F08BEF95F017A014
:1029C000E4EF94F0E6EF94F0ECEF94F0D890173049
:1029D0000109176EEEEF94F0D890173208A0F3EFCC
:1029E00094F0F5EF94F0F6EF94F0178E0B340B3271
:1029F0000A3209320832162A8BEF95F00C50085C27
:102A00000D5009580E500A580B50800A106E0F5086
:102A1000800A1058D8B00FEF95F011EF95F03CEF09
:102A200095F008500C5C106E09500D58116E0A504C
:102A30000E58126E0B500F58136EFF0E1024086EB6
:102A4000FF0E1120096EFF0E12200A6EFF0E1320DA
:102A50000B6E800E141A176C1750D8A432EF95F035
:102A600034EF95F044EF95F0010E0826000E092290
:102A70000A220B2244EF95F00C50085E0D50095AC3
:102A80000E500A5A0F500B5A085009100A100B101A
:102A9000D8A44DEF95F04FEF95F084EF95F01750D7
:102AA000D8A455EF95F057EF95F084EF95F0000E10
:102AB000086E000E096E000E0A6E000E0B6E1FEF00
:102AC00096F0D890083609360A360B3617AE6BEFFB
:102AD00095F06DEF95F06EEF95F0088017A073EF0D
:102AE00095F075EF95F079EF95F0D88017367BEF7C
:102AF00095F0D89017361650D8B481EF95F083EF43
:102B000095F084EF95F016060AAE89EF95F08BEFFD
:102B100095F061EF95F0000E156E17AE92EF95F0FF
:102B200094EF95F0ACEF95F017C010F07F0E1016F3
:102B3000D8B49DEF95F09FEF95F0A3EF95F0010EBF
:102B4000156EACEF95F008A0A8EF95F0AAEF95F000
:102B5000ACEF95F09FEF95F01550D8B4B2EF95F02B
:102B6000B4EF95F0DFEF95F0010E0826000E092274
:102B70000A220B220BA0BFEF95F0C1EF95F0DFEF1B
:102B800095F008C010F009C011F00AC012F00BC097
:102B900013F01334133212321132103210C008F015
:102BA00011C009F012C00AF013C00BF01628D8B4F7
:102BB000DCEF95F0DEEF95F0DFEF95F0162A1628A2
:102BC000D8B4E5EF95F0E7EF95F0EFEF95F01650FC
:102BD000D8A4EDEF95F0EFEF95F001EF96F0000E31
:102BE000086E000E096E000E0A6E000E0B6E165077
:102BF000D8A4FDEF95F0FFEF95F001EF96F0000EF1
:102C0000146E16A006EF96F008EF96F00BEF96F014
:102C10000A8E0CEF96F00A9ED89016300B6E14AE0A
:102C200014EF96F016EF96F017EF96F00B8E08C0A3
:102C300008F009C009F00AC00AF00BC00BF012003E
:102C40001950800B226E19501924286E18AE2BEFE4
:102C500096F02DEF96F02EEF96F028802850D8B4FD
:102C600034EF96F036EF96F049EF96F02828D8A486
:102C70003CEF96F03EEF96F046EF96F0000E166EA3
:102C8000000E176E000E186E000E196E188E51EFA2
:102C900096F0000E166E000E176E000E186E000EE7
:102CA000196E1D50800B221A1D501D24236E1CAE60
:102CB0005CEF96F05EEF96F05FEF96F02380235086
:102CC000D8B465EF96F067EF96F07AEF96F0232888
:102CD000D8A46DEF96F06FEF96F077EF96F0000EB8
:102CE0001A6E000E1B6E000E1C6E000E1D6E1C8EEA
:102CF00082EF96F0000E1A6E000E1B6E000E1C6E18
:102D0000000E1D6E2350D8B488EF96F08AEF96F02F
:102D100092EF96F02850D8A490EF96F092EF96F0AC
:102D20009CEF96F0000E166E000E176E000E186ED9
:102D3000000E196E46EF98F01C5016026F00CCFF83
:102D40002DF06F00D0FF2EF02D50246E256A266ADC
:102D5000276A2E50296E2A6A2B6A2C6A1B5017028A
:102D60006F00CCFF2DF06F00D0FF2EF02D502426E9
:102D7000000E2522262227222E502926000E2A2246
:102D80002B222C221A5018026F00CCFF2DF06F005E
:102D9000D0FF2EF02D502426000E25222622272299
:102DA0002E502926000E2A222B222C2226C027F064
:102DB00025C026F024C025F0246A1A5017026F009F
:102DC000CCFF2DF06F00D0FF2EF02D5024262E507A
:102DD0002522000E2622000E27221B5016026F000D
:102DE000CCFF2DF06F00D0FF2EF02D5024262E505A
:102DF0002522000E2622000E272226C027F025C0FD
:102E000026F024C025F0246A1A5016026F00CCFF69
:102E10002DF06F00D0FF2EF02D5024262E502522AD
:102E2000000E2622000E27221C5017026F00CCFF36
:102E30002DF06F00D0FF2EF02D5029262E502A2283
:102E4000000E2B22000E2C221B5018026F00CCFF0C
:102E50002DF06F00D0FF2EF02D5029262E502A2263
:102E6000000E2B22000E2C221C5018026F00CCFFEB
:102E70002DF06F00D0FF2EF02D501E6E2E501F6EC5
:102E8000206A216A20C021F01FC020F01EC01FF060
:102E90001E6A1E5029261F502A2220502B22215004
:102EA0002C2224C01EF025C01FF026C020F027C011
:102EB00021F0190E61EF97F0D890213220321F32A5
:102EC0001E32E82E5CEF97F01E5029261F502A2252
:102ED00020502B2221502C2226C027F025C026F07E
:102EE00024C025F0246A235028C01EF01F6A1E2625
:102EF000000E1F22820E1E242D6EFF0E1F202E6E2E
:102F000097EF97F0D89029362A362B362C3627AEF5
:102F10008CEF97F08EEF97F08FEF97F02980D89095
:102F200024362536263627362D06D8A02E062BAE7B
:102F30009CEF97F09EEF97F082EF97F0000E236ED4
:102F400027AEA5EF97F0A7EF97F0CBEF97F0FF0E26
:102F500024141E6EFF0E25141F6EFF0E2614206E05
:102F60007F0E2714216E1E501F1020102110D8B480
:102F7000BCEF97F0BEEF97F0C2EF97F0010E236E13
:102F8000CBEF97F029A0C7EF97F0C9EF97F0CBEF01
:102F900097F0BEEF97F02350D8B4D1EF97F0D3EF6E
:102FA00097F0F7EF97F0010E2926000E2A222B2228
:102FB0002C222CA0DEEF97F0E0EF97F0F7EF97F0E0
:102FC00029C01EF02AC01FF02BC020F02CC021F019
:102FD0002134213220321F321E321EC029F01FC080
:102FE0002AF020C02BF021C02CF02D4A2E2A2EBE14
:102FF00002EF98F02E5008E12D28D8A002EF98F0AB
:1030000004EF98F00EEF98F0000E296E000E2A6E75
:10301000800E2B6E7F0E2C6E3CEF98F02EBE1BEFB9
:1030200098F02E5006E12D04D8B019EF98F01BEF60
:1030300098F027EF98F0000E296E000E2A6E000E11
:103040002B6E000E2C6E000E226E3CEF98F02DC001
:1030500028F0FF0E2916FF0E2A167F0E2B16000EE3
:103060002C1628A036EF98F038EF98F039EF98F04A
:103070002B8ED89028302C6E22502C1229C016F09E
:103080002AC017F02BC018F02CC019F012003250D3
:10309000800B3F6E32503224466E31AE52EF98F0C4
:1030A00054EF98F055EF98F046804650D8B45BEF57
:1030B00098F05DEF98F072EF98F04628D8A463EF8F
:1030C00098F065EF98F06DEF98F0000E2F6E000EFF
:1030D000306E000E316E000E326E318E000E326E8A
:1030E0007AEF98F0000E2F6E000E306E000E316EEB
:1030F000000E326E3650800B3F1A36503624476E23
:1031000035AE85EF98F087EF98F088EF98F047801C
:103110004750D8B48EEF98F090EF98F0A5EF98F064
:103120004728D8A496EF98F098EF98F0A0EF98F081
:10313000000E336E000E346E000E356E000E366ECD
:10314000358E000E366EADEF98F0000E336E000E29
:10315000346E000E356E000E366E3350341035105E
:103160003610D8A4B6EF98F0B8EF98F0D0EF98F0FA
:10317000000E2F6E000E306E000E316E000E326E9D
:10318000800E31127F0E32123F5032122FC02FF0BC
:1031900030C030F031C031F032C032F013EF9AF06D
:1031A0004650D8A4D6EF98F0D8EF98F0E2EF98F018
:1031B000000E2F6E000E306E000E316E000E326E5D
:1031C00013EF9AF0475046C037F0386A375E000E6A
:1031D000385A7F0E3724406E000E3820416E2FC0C3
:1031E0003BF030C03CF031C03DF032C03EF0000E4C
:1031F0002F6E000E306E000E316E000E326E000E1D
:10320000426E000E436E000E446E000E456E000EC0
:10321000476E43EF99F04750D8B411EF99F013EF90
:1032200099F02AEF99F0D8903B363C363D363E3641
:10323000D8902F3630363136323645AE22EF99F0FF
:1032400024EF99F025EF99F02F80D890423643363D
:103250004436453633503B5C34503C5835503D582D
:1032600036503E58D8A037EF99F039EF99F042EF39
:1032700099F0458C33503B5E34503C5A35503D5AA2
:1032800036503E5A472A190E476449EF99F04BEFE2
:1032900099F00BEF99F03B503C103D103E10D8B424
:1032A00054EF99F056EF99F06EEF99F042806EEF7F
:1032B00099F0D8902F3630363136323645AE63EF3E
:1032C00099F065EF99F066EF99F02F80D89042362B
:1032D0004336443645364006D8A0410631AE73EF3A
:1032E00099F075EF99F059EF99F0000E476E45AEE1
:1032F0007CEF99F07EEF99F0A2EF99F0FF0E421467
:10330000376EFF0E4314386EFF0E4414396E7F0E75
:1033100045143A6E3750381039103A10D8B493EF3C
:1033200099F095EF99F099EF99F0010E476EA2EFA1
:1033300099F02FA09EEF99F0A0EF99F0A2EF99F0ED
:1033400095EF99F04750D8B4A8EF99F0AAEF99F00B
:10335000CEEF99F0010E2F26000E302231223222BC
:1033600032A0B5EF99F0B7EF99F0CEEF99F02FC0FA
:1033700037F030C038F031C039F032C03AF03A346A
:103380003A3239323832373237C02FF038C030F065
:1033900039C031F03AC032F0404A412A41BED9EF3B
:1033A00099F0415008E14028D8A0D9EF99F0DBEF1F
:1033B00099F0E6EF99F0000E416E4068000E2F6E16
:1033C000000E306E000E316E000E326E41BEF3EF15
:1033D00099F0415006E14004D8B0F1EF99F0F3EFD5
:1033E00099F001EF9AF0000E416E000E406E000E53
:1033F0002F6E000E306E000E316E000E326E000E1B
:103400003F6E40C046F046A008EF9AF00AEF9AF0EF
:103410000DEF9AF0318E0EEF9AF0319ED890463033
:10342000326EC4EF98F012005A0E086EFB0E096E51
:10343000D0ECB5F0AC0E0001F36F010EF46F000E8E
:103440000101AC6F470EAD6F3F0EAE6F400E000135
:10345000FC6F030EFB6FF3C01DF0F4C01EF0FBC049
:103460001FF0206AFC51ECECB4F06E0E086EF90E01
:10347000096ED0ECB5F0050E0101AC6F000EAD6F1A
:10348000140EAE6F400E0001FC6FAC0EF36F010E18
:10349000F46F030EFB6FF3C01DF0F4C01EF0FBC011
:1034A0001FF0206AFC51ECECB4F0F70E086EFA0E37
:1034B000096ED0ECB5F0060E0101AC6F800EAD6F59
:1034C000010EAE6F400E0001FC6FAC0EF36F010EEB
:1034D000F46F030EFB6FF3C01DF0F4C01EF0FBC0D1
:1034E0001FF0206AFC51ECECB4F05C0E086EFA0E92
:1034F000096ED0ECB5F0070E0101AC6F090EAD6F8F
:10350000600EAE6F400E0001FC6FAC0EF36F010E4B
:10351000F46F030EFB6FF3C01DF0F4C01EF0FBC090
:103520001FF0206AFC51ECECB4F0400E0001FC6F7F
:10353000000E0101AC6F000EAD6FAC0E0001F36F19
:10354000010EF46F040E1D6EF3C01EF0F4C01FF0E8
:10355000000E216E030E206EFC51BFECB1F0010194
:10356000AC510001F26FF16B0101AD510001F12589
:10357000FD6F0101000E0001F221FE6F200ED86FD9
:10358000020ED96F1A0EDA6FFD0EDB6FFDC0DCF094
:10359000FEC0DDF0FBECB5F0200E086E020E096EE9
:1035A00017ECB4F0400E0001FC6F000E0101AC6F8F
:1035B000000EAD6FAC0E0001F36F010EF46F070E3D
:1035C0001D6EF3C01EF0F4C01FF0000E216E030E3E
:1035D000206EFC51BFECB1F00101AC510001F26F63
:1035E000F16B0101AD510001F125FD6F0101000EEC
:1035F0000001F221FE6F6F0E1A6E120E1B6E030E8B
:103600001C6E410E1D6EFDC008F0FEC009F00A6A76
:103610000B6A000E3AECA3F008C016F009C017F0D0
:103620000AC018F00BC019F020EC96F016C02FF06D
:1036300017C030F018C031F019C032F0000E336EF0
:10364000000E346E000E356E470E366E47EC98F065
:103650002FC03AF130C03BF131C03CF132C03DF1F6
:10366000200E0001D86F020ED96FFA0EDA6FFC0E31
:10367000DB6F3AC1DCF03BC1DDF03CC1DEF03DC1A7
:10368000DFF0FBECB5F0200E086E020E096E17ECB1
:10369000B4F0400E0001FC6F000E0101AC6F000E93
:1036A000AD6F000EAE6FAC0E0001F36F010EF46F44
:1036B000FE0E1D6EF3C01EF0F4C01FF0000E216E52
:1036C000030E206EFC51BFECB1F00101AC510001C2
:1036D000F26FF16B0101AD510001F125FD6F0101A8
:1036E000000E0001F221FE6F200ED86F020ED96F7E
:1036F0008E0EDA6FFD0EDB6FFDC0DCF0FEC0DDF07C
:10370000FBECB5F0200E086E020E096E17ECB4F05B
:10371000400E0001FC6F000E0101AC6F000EAD6F9A
:10372000000EAE6FAC0E0001F36F010EF46FFF0ED2
:103730001D6EF3C01EF0F4C01FF0000E216E030ECC
:10374000206EFC51BFECB1F00101AC510001F26FF1
:10375000F16B0101AD510001F125FD6F0101000E7A
:103760000001F221FE6F200ED86F020ED96FA90E54
:10377000DA6FFD0EDB6FFDC0DCF0FEC0DDF0FBECB0
:10378000B5F0200E086E020E096E17ECB4F0B50EFF
:10379000086EFC0E096ED0ECB5F0120025C03DF0AD
:1037A00026C03EF027C03FF028C040F029C041F0BD
:1037B0002AC042F02BC043F02CC044F044BEE3EFDB
:1037C0009BF0E6EF9BF0010EE7EF9BF0000E3B6EE7
:1037D0003C6A3B503C10D8B4F0EF9BF0F2EF9BF00A
:1037E00002EF9CF0441E431E421E411E401E3F1E1F
:1037F0003E1E3D6C000E3E223F22402241224222CC
:103800004322442253BE07EF9CF009EF9CF00AEFDD
:103810009CF0549253BE17EF9CF0535006E15204B3
:10382000D8B015EF9CF017EF9CF01DEF9CF0000E48
:10383000386E010E376E21EF9CF052C037F053C046
:1038400038F06CC139F06DC13AF03B503C10D8A44F
:103850002CEF9CF02EEF9CF035EF9CF054A433EF4E
:103860009CF035EF9CF038EF9CF03906D8A03A0672
:10387000000E466E4F0E456E000E0201EF6FBDEF5B
:103880009CF04506D8A04606A00E4524D96E020E2F
:103890004620DA6E3DC008F03EC009F03FC00AF095
:1038A00040C00BF041C00CF042C00DF043C00EF020
:1038B00044C00FF00A0E106E000E116E000E126E54
:1038C000000E136E000E146E000E156E000E166EB6
:1038D000000E176E69ECA6F008C02DF009C02EF09E
:1038E0000AC02FF00BC030F00CC031F00DC032F028
:1038F0000EC033F00FC034F02DC01AF02FC01BF0F3
:10390000D9ECB7F01A50300FDF6E3706D8A0380662
:103910003906D8A03A063DC008F03EC009F03FC0C5
:103920000AF040C00BF041C00CF042C00DF043C0A3
:103930000EF044C00FF00A0E106E000E116E000E55
:10394000126E000E136E000E146E000E156E000E39
:10395000166E000E176EE6ECA4F008C03DF009C02C
:103960003EF00AC03FF00BC040F00CC041F00DC06B
:1039700042F00EC043F00FC044F046BEC8EF9CF0CA
:10398000465008E14504D8A0C8EF9CF0CAEF9CF06F
:10399000FAEF9CF03D503E103F1040104110421095
:1039A00043104410D8A4D7EF9CF0D9EF9CF041EF1E
:1039B0009CF038BEE6EF9CF0385006E13704D8B0F2
:1039C000E4EF9CF0E6EF9CF041EF9CF03ABEF1EFA3
:1039D0009CF03A5008E13904D8A0F1EF9CF0F3EFE5
:1039E0009CF0FAEF9CF054B2F8EF9CF0FAEF9CF0E8
:1039F00041EF9CF03B503C10D8A401EF9DF003EF49
:103A00009DF00AEF9DF054A408EF9DF00AEF9DF0A1
:103A100029EF9DF04506D8A046063B503C10D8A49F
:103A200014EF9DF016EF9DF01CEF9DF0000E366E2A
:103A30002B0E356E20EF9DF0000E366E2D0E356E7E
:103A4000A00E4524D96E020E4620DA6E6000D7F033
:103A5000DFFF23C018F024C019F0A00E45241A6E11
:103A6000020E46201B6E39C01CF03AC01DF099ECC6
:103A7000ADF018C023F019C024F0120053BE43EF7C
:103A80009DF045EF9DF046EF9DF0549253BE53EFED
:103A90009DF0535006E15204D8B051EF9DF053EF22
:103AA0009DF059EF9DF0000E376E010E366E5DEF02
:103AB0009DF052C036F053C037F06CC138F06DC184
:103AC00039F054A866EF9DF068EF9DF06CEF9DF023
:103AD000FE0E3826FF0E392225C03AF026C03BF0F4
:103AE00027C03CF028C03DF029C03EF02AC03FF07E
:103AF0002BC040F02CC041F0000E436E4F0E426EC2
:103B0000000E0201EF6F1FEF9EF04206D8A04306A1
:103B10000F0E3A14446E456A45BE98EF9DF045502D
:103B200009E10A0E445CD8A098EF9DF09AEF9DF051
:103B3000A2EF9DF0570E4424446E000E4520456EC2
:103B4000A8EF9DF0300E4424446E000E4520456ED3
:103B5000BF0E2E6EFF0E2F6E2D50306E316A2E501E
:103B600030262F503122315007E11A0E305CD8B088
:103B7000BCEF9DF0BEEF9DF0E1EF9DF09F0E2E6E2D
:103B8000FF0E2F6E200E4410306E000E4510316E69
:103B90002E5030262F503122315007E11A0E305C62
:103BA000D8B0D5EF9DF0D7EF9DF0E1EF9DF044C088
:103BB0000EF045C00FF054ECB7F00EC044F00FC04B
:103BC00045F0A00E4224D96E020E4320DA6E60004A
:103BD00013F1DFFF3606D8A037063806D8A039061D
:103BE0003AC02EF03BC02FF03CC030F03DC031F069
:103BF0003EC032F03FC033F040C034F041C035F039
:103C0000050E0CEF9EF0D89035323432333232321A
:103C1000313230322F322E32E82E03EF9EF02EC09A
:103C20003AF02FC03BF030C03CF031C03DF032C024
:103C30003EF033C03FF034C040F035C041F043BEE9
:103C40002BEF9EF0435009E1020E425CD8A02BEF0F
:103C50009EF02DEF9EF05DEF9EF03A503B103C1031
:103C60003D103E103F1040104110D8A43AEF9EF096
:103C70003CEF9EF085EF9DF037BE49EF9EF0375048
:103C800006E13604D8B047EF9EF049EF9EF085EF8D
:103C90009DF039BE54EF9EF0395008E13804D8A0A9
:103CA00054EF9EF056EF9EF05DEF9EF054B25BEF46
:103CB0009EF05DEF9EF085EF9DF054A862EF9EF0C0
:103CC00064EF9EF07BEF9EF04206D8A04306A00E64
:103CD0004224D96E020E4320DA6E6000B7F0DFFF97
:103CE0004206D8A04306A00E4224D96E020E4320FD
:103CF000DA6E300EDF6E23C018F024C019F0A00E6B
:103D000042241A6E020E43201B6E38C01CF039C0CC
:103D10001DF099ECADF018C023F019C024F012008A
:103D2000000E0001F76F030EF86F6000DFF3D9FF9C
:103D30006000E3F3DAFF000EDF6E3D017599738FCB
:103D4000000E0101E66F020EE56FE5C108F0E6C165
:103D500009F0A5ECB8F00009D8B4B1EF9EF0B3EFCC
:103D60009EF0C3EF9FF00101E635E6310001F16FEF
:103D70000101E5310001FD6FF1C0FEF0F7C0D8F0A0
:103D8000F8C0D9F0B90EDA6FFB0EDB6FE5C1DCF0DD
:103D9000E6C1DDF0FDC0DEF0FEC0DFF0FBECB5F00B
:103DA00064EF9FF0F7C016F0F8C017F0C30E186E5E
:103DB000FD0E196E28ECBAF0BBEF9FF0200E086ED6
:103DC000020E096E620E0A6EFF0E0B6E32ECB3F03D
:103DD000F7C008F0F8C009F077ECB5F008C0E3F1DF
:103DE00009C0E4F10101E3510001F7250C6E010166
:103DF000E4510001F8210D6E200E0E6E020E0F6EC2
:103E000086ECB4F0BBEF9FF0F7C016F0F8C017F0E7
:103E10003F0E186EFF0E196E28ECBAF0BBEF9FF044
:103E2000F7C016F0F8C017F0E20E186EFE0E196E0D
:103E300028ECBAF0BBEF9FF0F7C016F0F8C017F00F
:103E4000900E186EFF0E196E28ECBAF0BBEF9FF0C3
:103E5000F7C016F0F8C017F0500E186EFE0E196E6F
:103E600028ECBAF0BBEF9FF0F7C016F0F8C017F0DF
:103E7000730E186EFF0E196E28ECBAF0BBEF9FF0B0
:103E8000F7C016F0F8C017F0C10E186EFF0E196ECD
:103E900028ECBAF0BBEF9FF0F7C016F0F8C017F0AF
:103EA000720E186EFD0E196E28ECBAF0BBEF9FF083
:103EB000F7C016F0F8C017F0A90E186EFF0E196EB5
:103EC00028ECBAF0BBEF9FF0FDC0F1F0FEC0F2F0BD
:103ED0000001F251000AD8B470EF9FF058EF9FF044
:103EE000F151200AD8B4D2EF9EF0010AD8B4D2EF33
:103EF0009EF0030AD8B4D2EF9EF0010AD8B4D2EFF4
:103F00009EF0040AD8B4D2EF9EF00F0AD8B4DEEFC8
:103F10009EF0010AD8B4DEEF9EF0030AD8B4DEEFBB
:103F20009EF01D0AD8B404EF9FF00F0AD8B410EF2A
:103F30009FF0010AD8B410EF9FF0030AD8B410EF35
:103F40009FF0010AD8B410EF9FF0070AD8B41CEF15
:103F50009FF07C0AD8B428EF9FF0170AD8B434EF4A
:103F60009FF03F0AD8B440EF9FF0C80AD8B44CEF96
:103F70009FF058EF9FF0F7C008F0F8C009F017EC79
:103F8000B4F04EECB9F0020E0101E525E56F000E2C
:103F9000E621E66FE6BFD6EF9FF0E65109E1FC0EA1
:103FA000E55DD8A0D6EF9FF0D8EF9FF0A5EF9EF08B
:103FB0003D01739F75894EECB9F03D01738F12007E
:103FC000400E0001FC6F000E0101AC6F000EAD6FE2
:103FD000AC0E0001F36F010EF46F020E1D6EF3C004
:103FE0001EF0F4C01FF0000E216E030E206EFC5177
:103FF000BFECB1F00101AC51496E486AAD514824A3
:10400000746F000E4920756F400E0001FC6F000EAA
:104010000101AC6F000EAD6FAC0E0001F36F010E2D
:10402000F46F010E1D6EF3C01EF0F4C01FF0000E01
:10403000216E030E206EFC51BFECB1F00101AC51BA
:10404000496E486AAD514824766F000E4920776F5B
:10405000400E0001FC6F000E0101AC6F000EAD6F51
:10406000AC0E0001F36F010EF46F070E1D6EF3C06E
:104070001EF0F4C01FF0000E216E030E206EFC51E6
:10408000BFECB1F00101AC51496E486AAD51482412
:104090000001FD6F0101000E49200001FE6F6F0E4F
:1040A0001A6E120E1B6E030E1C6E410E1D6EFDC0AD
:1040B00008F0FEC009F00A6A0B6A000E3AECA3F0A1
:1040C00008C016F009C017F00AC018F00BC019F0AC
:1040D00020EC96F016C02FF017C030F018C031F069
:1040E00019C032F0000E336E000E346E000E356EC5
:1040F000470E366E47EC98F02FC03AF130C03BF1D6
:1041000031C03CF132C03DF1400E0001FC6F000EA9
:104110000101AC6F000EAD6FAC0E0001F36F010E2C
:10412000F46F060E1D6EF3C01EF0F4C01FF0000EFB
:10413000216E020E206EFC51BFECB1F00101AC51BA
:10414000496E486AAD514824706F000E4920716F66
:1041500070C148F071C149F0040E4A6ED8904932DE
:1041600048324A2EAEEFA0F048500F0B9F6F9F05CC
:10417000D8A4BDEFA0F0BFEFA0F0C0EFA0F0BA98B8
:10418000400E0001FC6F000E0101AC6F000EAD6F20
:10419000AC0E0001F36F010EF46F040E1D6EF3C040
:1041A0001EF0F4C01FF0000E216E030E206EFC51B5
:1041B000BFECB1F00101AC51496E486AAD514824E1
:1041C000726F000E4920736F400E0001FC6F000EED
:1041D0000101AC6F000EAD6FAC0E0001F36F010E6C
:1041E000F46F030E1D6EF3C01EF0F4C01FF0000E3E
:1041F000216E030E206EFC51BFECB1F00101AC51F9
:10420000496E486AAD5148240001FD6F0101000E5E
:1042100049200001FE6FFDC008F0FEC009F00A6AE7
:104220000B6A000E3AECA3F008C02FF009C030F082
:104230000AC031F00BC032F0000E336E400E346E07
:104240001C0E356E450E366E47EC98F02FC046F1C9
:1042500030C047F131C048F132C049F1120032C1DB
:1042600066F033C167F034C168F035C169F048C009
:1042700066F049C067F04AC068F04BC069F0810E33
:104280004C6EFF0E4D6E66C04EF067C04FF068C0BA
:1042900050F069C051F0180E53EFA1F0D890513290
:1042A00050324F324E32E82E4EEFA1F04E504C2499
:1042B0000001646F000E4D20656F65BF69EFA1F0CE
:1042C000655109E1170E645DD8A069EFA1F06BEFAD
:1042D000A1F075EFA1F048C048F049C049F04AC0CC
:1042E0004AF04BC04BF039EFA2F065BF7AEFA1F076
:1042F0007CEFA1F0EDEFA1F064C04CF0FF0E4D6E2D
:10430000FF0E4E6E7F0E4F6E000E506E4C668BEFA2
:10431000A1F093EFA1F0503450324F324E324D3273
:104320004C2E86EFA1F04DC060F04EC061F04FC042
:1043300062F050C063F00001605166154C6E61512F
:1043400067154D6E625168154E6E635169154F6E5B
:104350004C504D104E104F10D8A4B1EFA1F0B3EF58
:10436000A1F0B5EFA1F06BEFA1F066C04CF067C013
:104370004DF068C04EF069C04FF0200EC5EFA1F0BF
:10438000D8904F324E324D324C32E82EC0EFA1F071
:104390004C504D104E104F10D8B4D1EFA1F0D3EFC8
:1043A000A1F0DBEFA1F060516627615167236251F4
:1043B000682363516923601D4C6E611D4D6E621D43
:1043C0004E6E631D4F6E4C5066174D5067174E5022
:1043D00068174F50691731EFA2F066C04CF067C004
:1043E0004DF068C04EF069C04FF0200EFDEFA1F017
:1043F000D8904F324E324D324C32E82EF8EFA1F0C9
:104400004C504D104E104F10D8A409EFA2F00BEFF6
:10441000A2F015EFA2F0000E666F000E676F000E9F
:10442000686F000E696F31EFA2F0D89066354C6E60
:1044300067354D6E68354E6E69354F6E4C504D1078
:104440004E104F10D8B427EFA2F029EFA2F031EFB1
:10445000A2F0000E666F000E676F800E686FBF0ED1
:10446000696F66C048F067C049F068C04AF069C02B
:104470004BF0120053BE3FEFA2F041EFA2F042EF2B
:10448000A2F0549253BE4FEFA2F0535006E15204F3
:10449000D8B04DEFA2F04FEFA2F055EFA2F0000E12
:1044A000366E010E356E59EFA2F052C035F053C092
:1044B00036F06CC137F06DC138F025C039F026C038
:1044C0003AF027C03BF028C03CF029C03DF02AC09C
:1044D0003EF02BC03FF02CC040F0000E426E4F0E5D
:1044E000416E000E0201EF6FECEFA2F04106D8A082
:1044F0004206A00E4124D96E020E4220DA6E39C067
:1045000008F03AC009F03BC00AF03CC00BF03DC0D7
:104510000CF03EC00DF03FC00EF040C00FF00A0E90
:10452000106E000E116E000E126E000E136E000E55
:10453000146E000E156E000E166E000E176ECFEC88
:10454000ACF008C02DF009C02EF00AC02FF00BC04F
:1045500030F00CC031F00DC032F00EC033F00FC09F
:1045600034F02D50300FDF6E3506D8A036063706F2
:10457000D8A0380639C008F03AC009F03BC00AF0AC
:104580003CC00BF03DC00CF03EC00DF03FC00EF043
:1045900040C00FF00A0E106E000E116E000E126E6B
:1045A000000E136E000E146E000E156E000E166EC9
:1045B000000E176E15ECABF008C039F009C03AF0E8
:1045C0000AC03BF00BC03CF00CC03DF00DC03EF00B
:1045D0000EC03FF00FC040F041504210D8B4F3EF8E
:1045E000A2F0F5EFA2F025EFA3F039503A103B10FE
:1045F0003C103D103E103F104010D8A402EFA3F035
:1046000004EFA3F076EFA2F036BE11EFA3F0365020
:1046100006E13504D8B00FEFA3F011EFA3F076EF69
:10462000A2F038BE1CEFA3F0385008E13704D8A040
:104630001CEFA3F01EEFA3F025EFA3F054B223EF7D
:10464000A3F025EFA3F076EFA2F023C018F024C06A
:1046500019F0A00E41241A6E020E42201B6E37C0C4
:104660001CF038C01DF099ECADF018C023F019C053
:1046700024F01200106E1050D8B441EFA3F043EFB5
:10468000A3F065EFA3F00BBE4AEFA3F048EFA3F051
:1046900065EFA3F008C00CF009C00DF00AC00EF0E1
:1046A0000BC00FF00C1E0D1E0E1E0F1E0C2A000E4E
:1046B0000D220E220F220CC012F00DC013F00EC0FE
:1046C00014F00FC015F06DEFA3F008C012F009C090
:1046D00013F00AC014F00BC015F0085009100A10AE
:1046E0000B10D8A476EFA3F078EFA3F082EFA3F03D
:1046F000000E086E000E096E000E0A6E000E0B6EA4
:1047000013EFA4F0960E116E8CEFA3F0112AD8903F
:104710001532143213321232000E12140C6E000EC7
:1047200013140D6E000E14140E6EFE0E15140F6E83
:104730000C500D100E100F10D8A4A1EFA3F0A3EF92
:10474000A3F086EFA3F0B1EFA3F0112A010E122619
:10475000000E132214221522D8901532143213326F
:104760001232000E12140C6E000E13140D6E000E99
:1047700014140E6EFF0E15140F6E0C500D100E104B
:104780000F10D8A4C6EFA3F0C8EFA3F0A5EFA3F0D5
:10479000D0EFA3F01106D890123613361436153622
:1047A00014BED5EFA3F0D7EFA3F0DFEFA3F0020E16
:1047B0001160DDEFA3F0DFEFA3F0CAEFA3F011B0BB
:1047C000E4EFA3F0E6EFA3F0E7EFA3F0149ED89098
:1047D000113211C00CF00D6A0E6A0F6A0CC00FF096
:1047E0000E6A0D6A0C6A0C5012120D5013120E5004
:1047F00014120F5015121050D8B401EFA4F003EFAB
:10480000A4F00BEFA4F00BBE0AEFA4F008EFA4F0A5
:104810000BEFA4F0158E12C008F013C009F014C0FD
:104820000AF015C00BF0120020EECEF110EE16F0DB
:10483000060E6F006FFFE3FFE806FBE213C021F0F6
:1048400014C022F021502210D8A429EFA4F02BEF9D
:10485000A4F02FEFA4F0160E216E000E226E21C0E0
:1048600008F022C009F077ECB5F008C025F009C0C7
:1048700026F052C023F053C024F024BE42EFA4F02F
:1048800044EFA4F059EFA4F02550235C2450800A93
:10489000156E2650800A1558D8A051EFA4F053EF9A
:1048A000A4F055EFA4F059EFA4F023C025F024C0E4
:1048B00026F025C023F026C024F06CC11FF06DC186
:1048C00020F054B066EFA4F068EFA4F085EFA4F0F8
:1048D00076EFA4F0000E096E200E086E11C00AF0EB
:1048E00012C00BF08DECABF0254A262A1F50255C38
:1048F0002650800A156E2050800A1558D8A083EFE4
:10490000A4F085EFA4F06AEFA4F0000E1E6E000E76
:104910001D6EAEEFA4F0600087F0F6FF60008BF034
:10492000F7FF000EF86E1F0EF76403D00800F55075
:1049300007D06F00DBFFE9FF6F00DFFFEAFFEF50FA
:10494000156E1550086E096A11C00AF012C00BF0FE
:104950008DECABF0214A222A1D4A1E2A23501D5CF1
:104960001E50800A156E2450800A1558D8A0BBEF3F
:10497000A4F0BDEFA4F08BEFA4F054A0C2EFA4F01C
:10498000C4EFA4F0E1EFA4F0D2EFA4F0000E096EA2
:10499000200E086E11C00AF012C00BF08DECABF0C7
:1049A000254A262A1F50255C2650800A156E205065
:1049B000800A1558D8A0DFEFA4F0E1EFA4F0C6EF0D
:1049C000A4F025C011F026C012F01200000E196EDE
:1049D00017BEEFEFA4F0EDEFA4F001EFA5F0171E66
:1049E000161E151E141E131E121E111E106C000E14
:1049F0001122122213221422152216221722010E2E
:104A0000196E0FBE08EFA5F006EFA5F01AEFA5F09E
:104A10000F1E0E1E0D1E0C1E0B1E0A1E091E086CFC
:104A2000000E09220A220B220C220D220E220F2236
:104A3000010E191A20EE1AF0070EDE6AE806FDE2F2
:104A4000105011101210131014101510161017100A
:104A5000D8B42DEFA5F02FEFA5F081EFA5F0010E52
:104A6000186E3DEFA5F0D890103611361236133679
:104A70001436153616361736182A17AE42EFA5F03B
:104A800044EFA5F033EFA5F0D8901A361B361C364C
:104A90001D361E361F36203621361050085C115048
:104AA000095812500A5813500B5814500C581550EE
:104AB0000D5816500E5817500F58D8A062EFA5F099
:104AC00064EFA5F075EFA5F01050085E1150095A7B
:104AD00012500A5A13500B5A14500C5A15500D5AB2
:104AE00016500E5A17500F5A1A80D8901732163295
:104AF000153214321332123211321032182E44EFA2
:104B0000A5F01950D8B487EFA5F089EFA5F099EF7B
:104B1000A5F0211E201E1F1E1E1E1D1E1C1E1B1E5C
:104B20001A6C000E1B221C221D221E221F22202274
:104B300021221AC008F01BC009F01CC00AF01DC0D9
:104B40000BF01EC00CF01FC00DF020C00EF021C0F5
:104B50000FF01200000E186E000E176E000E166E8B
:104B6000000E156EB6EFA5F00F4A102A60003FF058
:104B7000F6FF600043F0F7FF000EF86E0800F550F6
:104B8000200AD8B4C6EFA5F0C8EFA5F0B4EFA5F0A1
:104B9000F70E116EFF0E126E60003FF0F6FF600020
:104BA00043F0F7FF000EF86E0800F550136E146A1C
:104BB0001150132612501422145009E1050E135CF3
:104BC000D8A0E5EFA5F0E7EFA5F0B4EFA5F0F1EF81
:104BD000A5F0000E166E010E156E0F4A102A2EEF6C
:104BE000A6F060003FF0F6FF600043F0F7FF000E14
:104BF000F86E0800F550116E126A1250000AD8B40F
:104C000004EFA6F02EEFA6F011502B0AD8B4EDEF6A
:104C1000A5F0060AD8B4E9EFA5F02EEFA6F017C06C
:104C200008F018C009F0000E0B6E0A0E0A6EEBECCD
:104C3000B9F060003FF0F6FF600043F0F7FF000EB0
:104C4000F86E0800F550085E000E095A300E082470
:104C5000176E000E0920186EEDEFA5F0D00E116E44
:104C6000FF0E126E60003FF0F6FF600043F0F7FFAA
:104C7000000EF86E0800F550136E146A11501326DA
:104C800012501422145009E10A0E135CD8A04BEF05
:104C9000A6F04DEFA6F00FEFA6F015501610D8A411
:104CA00054EFA6F056EFA6F064EFA6F017C011F08F
:104CB00018C012F0111E121E114A122A11C00FF054
:104CC00012C010F068EFA6F017C00FF018C010F077
:104CD0001200000E196E0FBE72EFA6F070EFA6F074
:104CE00084EFA6F00F1E0E1E0D1E0C1E0B1E0A1EBC
:104CF000091E086C000E09220A220B220C220D222A
:104D00000E220F22010E196E17BE8BEFA6F089EF4F
:104D1000A6F09BEFA6F0171E161E151E141E131EDE
:104D2000121E111E106C000E1122122213221422C8
:104D300015221622172210501110121013101410E1
:104D4000151016101710D8B4A8EFA6F0AAEFA6F009
:104D5000F2EFA6F0010E186EB8EFA6F0D89010365C
:104D60001136123613361436153616361736182AFB
:104D700017AEBDEFA6F0BFEFA6F0AEEFA6F0105055
:104D8000085C1150095812500A5813500B5814500F
:104D90000C5815500D5816500E5817500F58D8A0D3
:104DA000D4EFA6F0D6EFA6F0E6EFA6F01050085E1E
:104DB0001150095A12500A5A13500B5A14500C5AD7
:104DC00015500D5A16500E5A17500F5AD8901732C8
:104DD0001632153214321332123211321032182EAA
:104DE000BFEFA6F01950D8B4F8EFA6F0FAEFA6F08E
:104DF0000AEFA7F00F1E0E1E0D1E0C1E0B1E0A1E24
:104E0000091E086C000E09220A220B220C220D2218
:104E10000E220F2208C008F009C009F00AC00AF0EB
:104E20000BC00BF00CC00CF00DC00DF00EC00EF05E
:104E30000FC00FF0120008C00FF009C010F00AC038
:104E400011F00BC012F00C06D8A00D060C2806E1DC
:104E50000D28D8A42EEFA7F030EFA7F03DEFA7F074
:104E6000000E096E000E086EC3EFA7F00F4A102A5D
:104E7000114A122A0C06D8A00D0660003FF0F6FF7A
:104E8000600043F0F7FF000EF86E1F0EF76403D0CA
:104E90000800F55007D06F00DBFFE9FF6F00DFFF70
:104EA000EAFFEF500009D8B458EFA7F05AEFA7F087
:104EB0009EEFA7F0600047F0F6FF60004BF0F7FFB1
:104EC000000EF86E0800F5500009D8B46AEFA7F09C
:104ED0006CEFA7F09EEFA7F00C500D10D8B473EF55
:104EE000A7F075EFA7F09EEFA7F0600047F0F6FF80
:104EF00060004BF0F7FF000EF86E08006F00D4FF63
:104F00000EF060003FF0F6FF600043F0F7FF000E88
:104F1000F86E1F0EF76403D00800F55007D06F003D
:104F2000DBFFE9FF6F00DFFFEAFFEF500E18D8B498
:104F30009CEFA7F09EEFA7F036EFA7F060003FF0E0
:104F4000F6FF600043F0F7FF000EF86E1F0EF764E7
:104F500003D00800F55007D06F00DBFFE9FF6F00BA
:104F6000DFFFEAFFEF500E6E600047F0F6FF6000D3
:104F70004BF0F7FF000EF86E0800F5500E5C086E5F
:104F8000096AD8A009061200400E50ECB0F0030EDA
:104F90002D6E080E2C6E770EE82EFED72C2EFCD729
:104FA0002D2EFAD700F0000E2F6E000E2E6E2A0462
:104FB0002B10D8A4DEEFA7F0E0EFA7F0E8EFA7F002
:104FC000250E086EF60E096ED0ECB5F04EECB9F079
:104FD000000E316E000E306E2A042B10D8A4F3EFB1
:104FE000A7F0F5EFA7F026EFA8F030503110D8B4B5
:104FF000FCEFA7F0FEEFA7F026EFA8F0070E3014A5
:105000002C6E000E31142D6E2C502D10D8A40BEFE9
:10501000A8F00DEFA8F026EFA8F02EC02CF02FC0BE
:105020002DF0D8902C362D36D8902C362D36D890A1
:105030002C362D36250E2C24086EF60E2D20096EEA
:10504000D0ECB5F02E4A2F2A4EECB9F0A50E302444
:10505000F66EF40E3120F76EF86A000EF8220800A2
:10506000F550F8ECB2F02A042B10D8A43AEFA8F0CF
:105070003CEFA8F04BEFA8F0A50E3024F66EF40E2E
:105080003120F76EF86A000EF8220800F550EBECBC
:10509000B6F04EECB9F0304A312A315009E1400EF9
:1050A000305CD8A056EFA8F058EFA8F0ECEFA7F0CE
:1050B000800E50ECB0F0D00E2C6ECA0EE82EFED74B
:1050C0002C2EFCD71200F70E086EFF0E096ED0ECE6
:1050D000B5F0000E266E300E02ECB2F0680E2A6EAD
:1050E000E40EE82EFED72A2EFCD700D0320E70EC4C
:1050F000BAF0000E266E300E02ECB2F0150E2A6EDB
:10510000C60EE82EFED72A2EFCD700D0330E70EC48
:10511000BAF0000E266E300E02ECB2F0150E2A6EBA
:10512000C60EE82EFED72A2EFCD700D0340E70EC27
:10513000BAF0000E266E250E02ECB2F0150E2A6EA5
:10514000C60EE82EFED72A2EFCD700D0350E70EC06
:10515000BAF0010E266E280E02ECB2F0150E2A6E81
:10516000C60EE82EFED72A2EFCD700D0360E70ECE5
:10517000BAF0010E266E080E02ECB2F0150E2A6E81
:10518000C60EE82EFED72A2EFCD700D0370E70ECC4
:10519000BAF0010E266E010E02ECB2F0030E2B6E79
:1051A000080E2A6E770EE82EFED72A2EFCD72B2E5D
:1051B000FAD700F0380E70ECBAF0010E266E060E2B
:1051C00002ECB2F0150E2A6EC60EE82EFED72A2E7D
:1051D000FCD700D0390E70ECBAF0010E266E0C0E22
:1051E00002ECB2F0150E2A6EC60EE82EFED72A2E5D
:1051F000FCD700D0410E70ECBAF0120051ECBBF0BD
:105200000009D8B406EFA9F008EFA9F044EFA9F01F
:1052100015EFA9F0A6ECBBF090EFA9F0FCECBBF009
:1052200090EFA9F0000E90EFA9F018C113F019C18A
:1052300014F020EE09F102D828EFA9F00500FA6E6B
:10524000DE50FD6EDE50FE6EDE50FF6EFA50120034
:10525000156E166A1650000AD8B431EFA9F012EF95
:10526000A9F01550010AD8B412EFA9F0030AD8B476
:105270000AEFA9F0010AD8B40EEFA9F0070AD8B4D2
:1052800012EFA9F012EFA9F046ECBBF00009D8B478
:105290004CEFA9F04EEFA9F08FEFA9F001012951D1
:1052A000030B0009D8B457EFA9F059EFA9F065EF47
:1052B000A9F0010E156E2951030B166E1550165EDE
:1052C00029511618FC0B1618296F60008FF4D9FFAE
:1052D000600093F4DAFFDF50196E234B242B25076F
:1052E000D8A0260725512611D8A479EFA9F07BEF85
:1052F000A9F083EFA9F044ECB2F0156E1550176ECB
:10530000186A87EFA9F0000E186E030E176E17C00B
:105310001AF01950B9ECBBF01A5090EFA9F0030E37
:1053200012000A340B34116E1150D8A49AEFA9F070
:105330009CEFA9F0A6EFA9F0000E086E000E096E12
:10534000000E0A6E000E0B6E13EFAAF008C00CF0F0
:1053500009C00DF00AC00EF00BC00FF0200EB6EF22
:10536000A9F0D8900F320E320D320C32E82EB1EF88
:10537000A9F00C50106E0A8EFF0E0816FF0E0916CB
:10538000FF0E0A16000E0B16960E115E11BECDEF23
:10539000A9F0CBEFA9F0E3EFA9F01150800A970F25
:1053A000D8B0D5EFA9F0D7EFA9F0D9EFA9F09CEFCD
:1053B000A9F0D8900B320A3209320832113ED9EFE7
:1053C000A9F0FBEFA9F01F0E1164E9EFA9F0EBEFD4
:1053D000A9F0F3EFA9F09CEFA9F0D89008360936B0
:1053E0000A360B3611061150D8A4F9EFA9F0FBEFDD
:1053F000A9F0EDEFA9F01050D8B401EFAAF003EF37
:10540000AAF00BEFAAF00B1E0A1E091E086C000E74
:1054100009220A220B2208C008F009C009F00AC0BC
:105420000AF00BC00BF01200000E2F14376E000EA6
:105430003014386E800E3114396E7F0E32143A6E8D
:105440003750381039103A10D8A429EFAAF02BEFB2
:10545000AAF033EFAAF0000E2F6E000E306E000E91
:10546000316E000E326E000E3314376E000E34149F
:10547000386E800E3514396E7F0E36143A6E375002
:10548000381039103A10D8A448EFAAF04AEFAAF021
:1054900052EFAAF0000E336E000E346E000E356E21
:1054A000000E366E32AE57EFAAF059EFAAF062EF57
:1054B000AAF02F6C301ED8B0302A311ED8B0312A55
:1054C000800E325636AE67EFAAF069EFAAF072EF9F
:1054D000AAF0336C341ED8B0342A351ED8B0352A21
:1054E000800E3656000E2F1A000E301A000E311A9A
:1054F000800E321A000E331A000E341A000E351ABE
:10550000800E361A33502F5C345030583550315895
:1055100036503258D8B08FEFAAF091EFAAF094EF3E
:10552000AAF0D89095EFAAF0D880120036C112F0F8
:1055300037C113F038C114F039C115F008C012F0AA
:1055400009C013F00AC014F00BC015F012C00CF023
:1055500013C00DF014C00EF015C00FF0180EB6EF0A
:10556000AAF0D8900F320E320D320C32E82EB1EF85
:10557000AAF00C50106E116A10501110D8A4C3EF8D
:10558000AAF0C5EFAAF0E5EFAAF0D89012340C6E9D
:1055900013340D6E14340E6E15340F6E0C500D1046
:1055A0000E100F10D8A4D7EFAAF0D9EFAAF0DFEFB2
:1055B000AAF0000E096E020E086E14EFABF0000E9A
:1055C000096E030E086E14EFABF010281110D8A46A
:1055D000ECEFAAF0EEEFAAF010EFABF012C00CF077
:1055E00013C00DF014C00EF015C00FF0090ED890C6
:1055F0000C360D360E360F36E82EF7EFAAF00C50AB
:105600000D100E100F10D8B408EFABF00BEFABF08D
:10561000010E0CEFABF0000E086E096A14EFABF050
:10562000000E096E040E086E120020EE18F0070E30
:10563000DE6AE806FDE2105011101210131014106B
:10564000151016101710D8B428EFABF02AEFABF0F6
:105650007CEFABF0010E206E38EFABF0D890103637
:105660001136123613361436153616361736202AEA
:1056700017AE3DEFABF03FEFABF02EEFABF0D890B5
:10568000183619361A361B361C361D361E361F368E
:105690001050085C1150095812500A5813500B58FA
:1056A00014500C5815500D5816500E5817500F58CE
:1056B000D8A05DEFABF05FEFABF070EFABF0105048
:1056C000085E1150095A12500A5A13500B5A1450BE
:1056D0000C5A15500D5A16500E5A17500F5A188062
:1056E000D890173216321532143213321232113268
:1056F0001032202E3FEFABF018C008F019C009F0AF
:105700001AC00AF01BC00BF01CC00CF01DC00DF03D
:105710001EC00EF01FC00FF012000A500B10D8B4BC
:1057200094EFABF096EFABF09FEFABF00A500B109D
:10573000D8A49DEFABF09FEFABF0A4EFABF0085017
:1057400003ECBCF0F8EFABF020EE09F00A50D926DC
:105750000B50DA22DE50DE10D8B4B1EFABF0B3EF6D
:10576000ABF0CEEFABF020EE09F00A50D9260B508B
:10577000DA2210EE03F00A50E1260B50E222DE504E
:10578000E65CE650800A106EDE50800A1058D8B0F1
:10579000CCEFABF0CEEFABF0F8EFABF020EE03F0D8
:1057A0000A50D9260B50DA226F0078FF0CF06F00F8
:1057B00074FF0DF060002BF0D9FF60002FF0DAFFCE
:1057C0006F0078FF0EF06F0074FF0FF00C500E2486
:1057D000D96E0D500F20DA6E600023F0DFFF20EE4F
:1057E00003F00A50D9260B50DA22DE2A000EDD2201
:1057F00012002C502D10D8A400EFACF002EFACF04A
:1058000006EFACF0000E2D6E010E2C6E2C50575C86
:105810005850800A2F6E2D50800A2F58D8B013EFA1
:10582000ACF015EFACF019EFACF057C02CF058C04D
:105830002DF02A042B10D8A420EFACF022EFACF00E
:1058400026EFACF02C507F0F50ECB0F0020E2A186F
:105850002B10D8A42EEFACF030EFACF034EFACF05E
:105860002C50BF0F50ECB0F0030E2A182B10D8A408
:105870003CEFACF03EEFACF042EFACF02C50930FAD
:1058800050ECB0F0040E2A182B10D8A44AEFACF05C
:105890004CEFACF050EFACF02C50D30F50ECB0F01C
:1058A000150E2F6EC60EE82EFED72F2EFCD700D079
:1058B0002E50F8ECB2F0150E2F6EC60EE82EFED765
:1058C0002F2EFCD700D0120001016C516D11D8A40D
:1058D0006CEFACF06EEFACF074EFACF06CC117F0A5
:1058E0006DC118F07AEFACF0FF0E6C25176EFF0E4D
:1058F0006D21186E54A07FEFACF081EFACF08AEF11
:10590000ACF013C008F0096A11C00AF012C00BF025
:105910008DECABF018BE8FEFACF091EFACF093EFE5
:10592000ACF097EFACF0000E186E000E176E000E84
:10593000166E000E156EA9EFACF0000E096E200E6B
:10594000086E11C00AF012C00BF08DECABF0154AD6
:10595000162A1750155C1650800A146E1850800ACB
:105960001458D8A0B6EFACF0B8EFACF09DEFACF0A7
:1059700054B0BDEFACF0BFEFACF0C8EFACF013C06B
:1059800008F0096A11C00AF012C00BF08DECABF000
:10599000010E1524116E000E1620126E120010500A
:1059A0001110121013101410151016101710D8B46F
:1059B000DCEFACF0DEEFACF026EFADF0010E186ED0
:1059C000ECEFACF0D8901036113612361336143690
:1059D000153616361736182A17AEF1EFACF0F3EF7E
:1059E000ACF0E2EFACF01050085C115009581250C6
:1059F0000A5813500B5814500C5815500D58165087
:105A00000E5817500F58D8A008EFADF00AEFADF0C0
:105A10001AEFADF01050085E1150095A12500A5A90
:105A200013500B5A14500C5A15500D5A16500E5A4A
:105A300017500F5AD89017321632153214321332CB
:105A4000123211321032182EF3EFACF008C008F009
:105A500009C009F00AC00AF00BC00BF00CC00CF032
:105A60000DC00DF00EC00EF00FC00FF01200000EB2
:105A70000D6E0BBE40EFADF03EEFADF046EFADF07A
:105A80000A6C0B1ED8B00B2A010E0D6E09BE4DEF2D
:105A9000ADF04BEFADF053EFADF0086C091ED8B090
:105AA000092A010E0D1A000E0F6E000E0E6E0A501E
:105AB0000B10D8B45EEFADF060EFADF088EFADF055
:105AC000010E0C6E68EFADF0D8900A360B360C2A3A
:105AD0000BAE6DEFADF06FEFADF064EFADF0D890C1
:105AE0000E360F360A50085C0B500958D8A07BEFD1
:105AF000ADF07DEFADF082EFADF00A50085E0B50D7
:105B0000095A0E80D8900B320A320C2E6FEFADF08E
:105B10000D50D8B48EEFADF090EFADF094EFADF046
:105B20000E6C0F1ED8B00F2A0EC008F00FC009F07F
:105B3000120054A09EEFADF0A0EFADF0AAEFADF0D3
:105B40001AC011F01BC012F018C013F019C014F0E5
:105B500076ECB7F01DBEAFEFADF0B1EFADF0B7EF43
:105B6000ADF01CC021F01DC022F0BBEFADF0000E67
:105B7000226E000E216E000E206E000E1F6ECDEF05
:105B8000ADF0000E096E200E086E18C00AF019C0A4
:105B90000BF08DECABF01F4A202A21501F5C2050E7
:105BA000800A1E6E2250800A1E58D8A0DAEFADF08F
:105BB000DCEFADF0C1EFADF054B0E1EFADF0E3EFED
:105BC000ADF0EDEFADF01AC011F01BC012F018C02F
:105BD00013F019C014F076ECB7F01AC008F01BC02F
:105BE00009F077ECB5F021500824186E22500920F6
:105BF000196E12002E6E2A50D8A401EFAEF003EFFA
:105C0000AEF005EFAEF0010E2A6E2A502B6E2C6A14
:105C10002B50575C5850800A2D6E2C50800A2D58FE
:105C2000D8B015EFAEF017EFAEF019EFAEF05704A5
:105C30002A6E2E04D8A41FEFAEF021EFAEF025EFB0
:105C4000AEF02A507F0F50ECB0F0020E2E18D8A400
:105C50002CEFAEF02EEFAEF032EFAEF02A50BF0FC9
:105C600050ECB0F0030E2E18D8A439EFAEF03BEF95
:105C7000AEF03FEFAEF02A50930F50ECB0F0040EB0
:105C80002E18D8A446EFAEF048EFAEF04CEFAEF0D1
:105C90002A50D30F50ECB0F0150E2B6EC60EE82E26
:105CA000FED72B2EFCD700D01200000EBA6E000ECD
:105CB000BB6E000EBC6EEF0EC26E9E0EC36E810EEA
:105CC000C46E660E3A01606F610E506F000E406F39
:105CD000000E816F000E516F000E416F000E616F5C
:105CE000C49ABC9AC296BA964099C298C298BA9879
:105CF000C480000E456F000E466F000E476F000E09
:105D0000656F010E666F000E676F000E5A6F000E12
:105D10005B6F000E6A6F000E6B6F000E426F000E1D
:105D2000526F180E626F436953696369446954691D
:105D30006469080E846F090E126F0A0E116F0B0E44
:105D40000D6F0C0E086F140EE26F210E136F220EF2
:105D5000146F130E166F170EE56F130EE16F12001E
:105D6000000E0D6E09BEB9EFAEF0B7EFAEF0BFEFAB
:105D7000AEF0086C091ED8B0092A010E0D6E0BBEDC
:105D8000C6EFAEF0C4EFAEF0CAEFAEF00A6C0B1E79
:105D9000D8B00B2A0A500B10D8B4D1EFAEF0D3EF25
:105DA000AEF0F7EFAEF0010E0C6EDBEFAEF0D89078
:105DB0000A360B360C2A0BAEE0EFAEF0E2EFAEF097
:105DC000D7EFAEF00A50085C0B500958D8A0EBEFA3
:105DD000AEF0EDEFAEF0F1EFAEF00A50085E0B5012
:105DE000095AD8900B320A320C2EE2EFAEF00D5069
:105DF000D8B4FDEFAEF0FFEFAEF003EFAFF0086CFC
:105E0000091ED8B0092A08C008F009C009F012001C
:105E1000000E0814106E000E0914116E800E0A1484
:105E2000126E7F0E0B14136E1050111012101310FF
:105E3000D8A41DEFAFF01FEFAFF027EFAFF0000ECB
:105E4000086E000E096E000E0A6E000E0B6E000E3C
:105E50000C14106E000E0D14116E800E0E14126EC6
:105E60007F0E0F14136E1050111012101310D8A4BF
:105E70003CEFAFF03EEFAFF046EFAFF0000E0C6E30
:105E8000000E0D6E000E0E6E000E0F6E0C500818F8
:105E90000FE10D5009180CE10E500A1809E10F50DE
:105EA0000B18D8B456EFAFF058EFAFF05BEFAFF090
:105EB000D8905CEFAFF0D8801200086E010E096E2A
:105EC000010129B766EFAFF068EFAFF0ADEFAFF0CB
:105ED00008C022F129952987FC0E29170F0E276F7C
:105EE000010E216FF40E206F2989000E006F780ECD
:105EF000016F010E026F000E126F000E136F000E85
:105F0000036F780E046F010E056F000E146F000E04
:105F1000156F000E066F780E076F010E086F000EEA
:105F2000166F000E176F000E096F780E0A6F010EC4
:105F30000B6F000E186F000E196FFC0E0C6F770EB2
:105F40000D6F010E0E6F000E1A6F000E1B6FD8EC56
:105F5000BBF065ECB9F0000E096E095012000101AA
:105F60002989D3EFAFF0EBECBBF0080E00EFB0F0F7
:105F7000EBECBBF0070E00EFB0F001012529BEEC01
:105F8000BBF0040E00EFB0F0070E01012719D8B4E2
:105F9000CCEFAFF0CEEFAFF0D0EFAFF0EEECBBF068
:105FA0000F0E00EFB0F012C113F013C114F002D8BD
:105FB000E4EFAFF00500FA6E0051FD6E0151FE6E88
:105FC0000251FF6EFA501200156E166A1650000A42
:105FD000D8B4EDEFAFF0C4EFAFF01550010AD8B46C
:105FE000C4EFAFF0030AD8B4B8EFAFF0010AD8B4E9
:105FF000B3EFAFF0070AD8B4BDEFAFF0C4EFAFF026
:1060000012005CECBBF00009D8A409EFB0F00BEF74
:10601000B0F00EEFB0F0040E4FEFB0F001012951D7
:10602000030B0009D8B417EFB0F019EFB0F025EF6B
:10603000B0F0010E176E2951030B186E1750185E41
:1060400029511818FC0B1818296F2507D8A0260706
:1060500025512611D8B42FEFB0F031EFB0F03FEF5B
:10606000B0F0E8ECBBF060008FF4D9FF600093F46F
:10607000DAFFDF6E0101234B242B0BEFB0F0AFEC06
:10608000AFF0196EE8ECBBF060008FF4D9FF600050
:1060900093F4DAFFDF6E0101234B242B1950120019
:1060A000286E2850F00B0C09296E29C022F000013F
:1060B000FC5100ECBAF0AAECB9F02850F00B08093A
:1060C000296E29C022F00001FC5100ECBAF0AAECC4
:1060D000B9F028C026F00F0E26162638F00B0C0952
:1060E000296E29C022F00001FC5100ECBAF0AAECA4
:1060F000B9F028C026F00F0E26162638F00B080936
:10610000296E29C022F00001FC5100ECBAF0AAEC83
:10611000B9F02804D8A48FEFB0F091EFB0F09DEF64
:10612000B0F0090E276E1E0E266EE40EE82EFED786
:10613000262EFCD7272EFAD700D012003901A3A7AC
:10614000A4EFB0F0A6EFB0F0EAEFB0F093A7ABEF9A
:10615000B0F0ADEFB0F0EAEFB0F06F00A0F7ABF148
:106160000D0E0101AB19D8B4B8EFB0F0BAEFB0F032
:10617000C5EFB0F08B5109E1800E8A5DD8A0C3EF66
:10618000B0F0C5EFB0F0DBEFB0F0010EA76F800EFE
:106190008A25D96E030E8B21DA6E000EDF6E8AC15E
:1061A0008CF18BC18DF1000E8B6F000E8A6F39015F
:1061B0009397EAEFB0F0800E8A25D96E030E8B21FB
:1061C000DA6E6000AFF6DFFF8A4B8B2B8AC18CF151
:1061D0008BC18DF11100260EF66E730EF76E010E57
:1061E000F86E00EEB6F110EE2DF009006F00D7FF4B
:1061F000EEFFE550E150F9E1040EF66E780EF76E11
:10620000010EF86E09006F00D4FF57F009006F000F
:10621000D4FF58F000EE00F310EE00F1EE6AE55006
:10622000E150FCE1E250FAE100EE00F2F00EEE6A1D
:10623000E806FDE100EE00F1B60EEE6AE806FDE1CB
:1062400000EEF3F00C0EEE6AE806FDE1566A556AC0
:10625000546A536A526A080ED56E000ED66E000E4E
:10626000D76E000100EF80F00D6E085009100A1083
:10627000D8B43DEFB1F03FEFB1F060EFB1F00D50A9
:10628000030D000EF324D96E010EF420DA6E6000C7
:1062900023F0DEFF600027F0DEFF60002BF0DEFF62
:1062A0000D50020D120EF324D96E010EF420DA6E99
:1062B00060002FF0DEFF600033F0DDFF7AEFB1F019
:1062C0000D50030D000EF324D96E010EF420DA6E8A
:1062D000000EDE6E780EDE6E010EDE6E0D50020DCB
:1062E000120EF324D96E010EF420DA6E000EDE6E6B
:1062F000000EDD6E1200000E2D6E000E2C6E97EF5C
:10630000B1F02C5028242A6E2D5029202B6E6000CD
:10631000ABF0F6FF6000AFF0F7FF000EF86E08007C
:10632000F550F8ECB2F02C4A2D2AAAECB9F02C501A
:1063300028242A6E2D5029202B6E6000ABF0F6FF2A
:106340006000AFF0F7FF000EF86E0800F55000098E
:10635000D8B4ADEFB1F0AFEFB1F0BEEFB1F0575040
:106360002C5C2D50800A2A6E5850800A2A58D8A0DA
:10637000BCEFB1F0BEEFB1F081EFB1F01200226ED0
:106380001EC025F01FC026F020C023F021C024F03D
:1063900022505DECAFF00009D8B4D1EFB1F0D3EFEB
:1063A000B1F0C8EFB1F03E0E0E6E6D0E0F6E010E25
:1063B000106E230E116E000E126ED7ECBAF01D0E89
:1063C000086E000E096E000E0B6E010E0A6E4DEC8B
:1063D000BAF0000E0E6E000E0F6E000E106E000E64
:1063E000116E000E126EC9ECBAF0C8ECBBF0C0EC36
:1063F000B9F0E806D8B4FFEFB1F001EFB2F0F7EF73
:10640000B1F01200286E2850F00B0C09296E29C03B
:1064100022F00001FC5100ECBAF0AAECB9F02850CF
:10642000F00B0809296E29C022F00001FC5100EC94
:10643000BAF0AAECB9F02604D8A421EFB2F023EF09
:10644000B2F043EFB2F028C027F00F0E271627381E
:10645000F00B0C09296E29C022F00001FC5100EC60
:10646000BAF0AAECB9F028C027F00F0E271627388B
:10647000F00B0809296E29C022F00001FC5100EC44
:10648000BAF0AAECB9F012000101298959EFB2F073
:10649000EBECBBF0070E82EFB2F001012529BEEC58
:1064A000BBF0030E82EFB2F0EEECBBF00A0E82EF0F
:1064B000B2F012C113F013C114F002D86AEFB2F0B7
:1064C0000500FA6E0051FD6E0151FE6E0251FF6E25
:1064D000FA501200156E166A1650000AD8B473EFFF
:1064E000B2F054EFB2F01550010AD8B454EFB2F044
:1064F000030AD8B448EFB2F0060AD8B44DEFB2F0B0
:1065000054EFB2F01200D8ECBBF0020E0101286F7C
:1065100096EFB2F0A6ECBBF0BDEFB2F0FCECBBF036
:10652000BDEFB2F090ECBBF0BDEFB2F014C113F0D0
:1065300015C114F020EE03F102D8A9EFB2F0050066
:10654000FA6EDE50FD6EDE50FE6EDE50FF6EFA50CB
:106550001200156E166A1650000AD8B4B2EFB2F0E7
:1065600092EFB2F01550020AD8B48AEFB2F0010AE5
:10657000D8B48EEFB2F092EFB2F012003901A3A7B7
:10658000C4EFB2F0C6EFB2F0C9EFB2F06F00A0F7FF
:10659000ABF1000E096E000E086E800E0824D96E55
:1065A000030E0920DA6E000EDF6E084A092A095030
:1065B00009E17F0E085CD8A0E0EFB2F0E2EFB2F0A4
:1065C000CDEFB2F03D01F289000EF96F000EFA6FC7
:1065D000000E0301806F000E01018D6F000E8C6FA5
:1065E000000EAB6F000EA76F3901938D93871200D9
:1065F000276E2750F00B0D09566E56C022F0000191
:10660000FC5100ECBAF0AAECB9F02750F00B0909E4
:10661000566E56C022F00001FC5100ECBAF0AAEC14
:10662000B9F027C026F00F0E26162638F00B0D09FC
:10663000566E56C022F00001FC5100ECBAF0AAECF4
:10664000B9F027C026F00F0E26162638F00B0909E0
:10665000566E56C022F00001FC5100ECBAF0AAECD4
:10666000B9F0120060002BF0F6FF60002FF0F7FF8A
:10667000000EF86E08006F00D4FF9CF159EFB3F0E4
:1066800060002BF0F6FF60002FF0F7FF000EF86EB1
:1066900008006F00D4FF9CF1600023F0D9FF600078
:1066A00027F0DAFF600073F6DFFF084A092A0A4A7A
:1066B0000B2A01019C51D8A460EFB3F062EFB3F054
:1066C00040EFB3F0600023F0D9FF600027F0DAFF5D
:1066D000000EDF6E1200D2C0D6F0D3C0D7F0000E8D
:1066E00001016B6F000E6A6F8DEFB3F0D0C0A8F0A0
:1066F000D1C0A9F0D60E0001AA6F000EAB6FD4C0B6
:10670000ACF0D5C0ADF0DCEC8DF00001A85101017A
:106710006A270001A95101016B2360005BF3F6FFBA
:1067200060005FF3F7FF000EF86E0800F5500009F7
:10673000D8A49DEFB3F09FEFB3F076EFB3F06AC14A
:10674000D0F06BC1D1F0120076ECB6F00101295106
:10675000030B0009D8B4AFEFB3F0B1EFB3F0BEEF65
:10676000B3F051ECBBF00009D8B4B9EFB3F0BBEF14
:10677000B3F0BEEFB3F0100E0101276F01012751F6
:10678000030DE50EF324F66EF40EF420F76EF86AAE
:10679000000EF82202D8DAEFB3F00500FA6E090015
:1067A000F550FD6E0900F550FE6E0900F550FF6EC4
:0A67B000FA5012000101276F1200D9
:1067BC003901A0AFE4EFB3F0E6EFB3F016EFB4F0AD
:1067CC006E009CF905F0000E066EA3A9F0EFB3F075
:1067DC00F2EFB3F0EBEFB3F005BEF7EFB3F0F9EF78
:1067EC00B3F0FFEFB3F0000E046E2E0E036E03EF4A
:1067FC00B4F0000E046E310E036E60000FF0EAFD73
:10680C00D8900536062A070E06640FEFB4F011EF88
:10681C00B4F0EBEFB3F0000E3A01676F3901A09FB3
:10682C001100000E0B6E000E0A6E40EFB4F0390131
:10683C00A3A923EFB4F025EFB4F01DEFB4F00A5088
:10684C000824D96E0B500920DA6EDF503D01EA6F37
:10685C000A4A0B2A0BBE3CEFB4F00B5009E1810E37
:10686C000A5CD8A03CEFB4F03EEFB4F040EFB4F0CB
:10687C004EEFB4F00A500824D96E0B500920DA6E92
:10688C00DF50D8A44CEFB4F04EEFB4F01DEFB4F0E1
:10689C001200FC0E01012917020E286F29955EEFDC
:1068AC00B4F0FAECBBF085EFB4F00F0E85EFB4F05A
:1068BC0016C113F017C114F020EE06F102D871EFD7
:1068CC00B4F00500FA6EDE50FD6EDE50FE6EDE504A
:1068DC00FF6EFA501200156E166A1650000AD8B4E4
:1068EC007AEFB4F05BEFB4F01550020AD8B457EF5E
:1068FC00B4F0010AD8B457EFB4F05BEFB4F0120067
:10690C000EC012F00FC013F00CC014F00DC015F037
:10691C001250106E1350116E124A132A600043F07D
:10692C00F6FF600047F0F7FF000EF86E600053F0C2
:10693C00D9FF600057F0DAFF144A152A1F0EF764CE
:10694C0003D00800F55007D06F00DBFFE9FF6F00A4
:10695C00DFFFEAFFEF50DF6EDF50D8A4B8EFB4F0E2
:10696C00BAEFB4F08EEFB4F01200000E2C6E000EE5
:10697C002B6ECEEFB4F02B502824D96E2C5029203E
:10698C00DA6EDF50F8ECB2F0AAECB9F02B4A2C2AF4
:10699C002B502824D96E2C502920DA6EDF50D8B415
:1069AC00DAEFB4F0DCEFB4F0EBEFB4F057502B5C53
:1069BC002C50800A2A6E5850800A2A58D8A0E9EF29
:1069CC00B4F0EBEFB4F0C1EFB4F01200216E215033
:1069DC005DECAFF00009D8B4F6EFB4F0F8EFB4F01A
:1069EC00EDEFB4F01DC008F01EC009F01FC00AF096
:1069FC0020C00BF04DECBAF0000E0E6E000E0F6EB8
:106A0C00000E106E000E116E000E126EC9ECBAF074
:106A1C00C8ECBBF0C0ECB9F0E806D8B418EFB5F090
:106A2C001AEFB5F010EFB5F01200000E3E01DE6F5C
:106A3C00000EDF6F000EE06F000EE16F000EE46FD2
:106A4C00000EE56F000EEA6F000EEC6F000EF16F9A
:106A5C00000EF36F000EF46F000EF56F000EF66F64
:106A6C00000EF76F000EF96F000EFA6F000EFB6F41
:106A7C00000EFC6F000EFD6F000EFE6F030EFF6F1D
:106A8C00840EF86F12003901A3A14FEFB5F051EF4E
:106A9C00B5F053EFB5F076EFB5F0A2AF58EFB5F017
:106AAC005AEFB5F05CEFB5F076EFB5F03D0179A596
:106ABC0062EFB5F064EFB5F066EFB5F076EFB5F0D8
:106ACC0079AF6BEFB5F06DEFB5F06FEFB5F076EF2A
:106ADC00B5F076A974EFB5F076EFB5F049EFB5F0F7
:106AEC00120008C00AF009C00BF07FEFB5F0084A9D
:106AFC00092A600023F0F6FF600027F0F7FF000E74
:106B0C00F86E1F0EF76403D00800F55007D06F0025
:106B1C00DBFFE9FF6F00DFFFEAFFEF500009D8A4AD
:106B2C009AEFB5F09CEFB5F07DEFB5F00A50085C2C
:0A6B3C00086E0B500958096E120094
:106B48006F00E8FF01F06F00ECFF02F03901A39F2E
:106B58000101EF51B76E6000BBF7B6FFEB51EC11C6
:106B6800ED11D8B4BAEFB5F0BCEFB5F0C9EFB5F098
:106B780002D8C9EFB5F00500FA6EEB51FD6EEC5185
:106B8800FE6EED51FF6EFA50120060000BF0FBFF35
:106B9800600007F0FAFF1100E8EFB5F03901A3A98A
:106BA800D8EFB5F0DAEFB5F0D2EFB5F0600023F02A
:106BB800F6FF600027F0F7FF000EF86E08006F0080
:106BC800D7FFEAFD084A092A600023F0F6FF6000B3
:106BD80027F0F7FF000EF86E0800F5500009D8A45A
:106BE800F8EFB5F0FAEFB5F0D2EFB5F01200DC0E21
:106BF8000001E46F000EE56FD8C0E6F0D9C0E7F0F9
:106C0800000EEA6F000EE96F000EF06F000EEF6FD6
:106C1800E60ED06F000ED16FDAC0D2F0DBC0D3F031
:106C2800E40ED46F000ED56F6BECB3F00001E951A0
:106C3800D825D96EEA51D921DA6E000EDF6E12001E
:106C4800010E0E6E200E08180910D8B42EEFB6F0FB
:106C580030EFB6F049EFB6F0F70E0A6EFF0E0B6E86
:106C680008C00CF009C00DF00A500C260B500D227C
:106C78000D5009E1050E0C5CD8A045EFB6F047EFC2
:106C8800B6F049EFB6F0000E0E6E0EC008F0096AB5
:106C980012001B6E010E1C6E010129B556EFB6F0ED
:106CA80058EFB6F074EFB6F02985000E1C6E25512A
:106CB800BEECBBF01B50D8B464EFB6F066EFB6F08C
:106CC8006DEFB6F0040E0101276F7CECB9F072EF9E
:106CD800B6F0030E0101276F3BECBBF080ECBAF075
:106CE8001C5012007DECBBF00009D8B47EEFB6F062
:106CF80080EFB6F084EFB6F0F7ECBBF09EEFB6F09D
:106D080067ECBBF00009D8B48CEFB6F08EEFB6F0A4
:106D180092EFB6F0F1ECBBF09EEFB6F072ECBBF080
:106D28000009D8B49AEFB6F09CEFB6F09EEFB6F033
:106D3800F4ECBBF0120020EE02F01350D9261450E8
:106D4800DA226F0078FF08F06F0074FF09F0600026
:106D58004FF0D9FF600053F0DAFF6F0078FF0AF0B8
:106D68006F0074FF0BF04DECBAF0000E0E6E000EC3
:106D78000F6E000E106E000E116E000E126ED7EC24
:106D8800BAF0020E1200000E3D01EC6F000EED6F1E
:106D9800000EEE6F000EEF6F000EF06F000EF16F39
:106DA800B00EF26F800EF36F000EF46F8A0EF56F5F
:106DB800000EF66F000EF76F000EF86F000EF96FF9
:106DC800000EFA6FF28BF289390193971200096E5F
:106DD800800E0A6E05EFB7F009500A140009D8B4FE
:106DE800F8EFB6F0FAEFB6F0FFEFB6F02A0E70EC57
:106DF800BAF002EFB7F0200E70ECBAF0D8900A3073
:106E08000A6E0A50D8A40BEFB7F00DEFB7F0F0EF09
:106E1800B6F01200BF0E106EFF0E116E0EC012F00B
:106E28000FC013F01050122611501322135007E10F
:106E38001A0E125CD8B023EFB7F025EFB7F02CEF9D
:106E4800B7F0200E0E100E6E0F500F6E30EFB7F029
:106E58000EC00EF00FC00FF01200000E331A000E15
:106E6800341A000E351A800E361A2FC008F030C0BA
:106E780009F031C00AF032C00BF033C00CF034C056
:106E88000DF035C00EF036C00FF0C0EC93F008C01E
:106E98002FF009C030F00AC031F00BC032F01200F8
:106EA8009F0E106EFF0E116E0EC012F00FC013F081
:106EB8001050122611501322135007E11A0E125CBB
:106EC800D8B069EFB7F06BEFB7F071EFB7F05F0EBE
:106ED8000E140E6E0F6A75EFB7F00EC00EF00FC0ED
:106EE8000FF01200000E176E000E166E87EFB7F047
:106EF80015C008F0096A13C00AF014C00BF08DEC35
:106F0800ABF0164A172A16501124D96E17501220C2
:106F1800DA6EDF50156E1550D8A495EFB7F097EFDD
:106F2800B7F07CEFB7F01200430EB96EEB0EB76EF8
:106F3800000EB66EB6506F00DCFE0BF00C6A0BC08C
:106F48000CF00B6A0B100101EE6F0C50EF6F39015A
:106F5800A39F938F0A0E086E780E096E010E0A6EB3
:106F680098ECBBF0900EB86E1200D29ED28AD29ED8
:106F7800D29CD28A550ED46EAA0ED46ED490000E2E
:106F8800D76E000ED66E080ED56E550ED46EAA0EAC
:106F9800D46ED4803901838781818491839F8495BD
:106FA800809FD29CD29ED29E12001BBEE6EFB7F005
:106FB8001B5006E11A04D8B0E4EFB7F0E6EFB7F0DB
:106FC800F4EFB7F01AC01CF01BC01DF01C1E1D1EEC
:106FD8001C4A1D2A1CC01AF01DC01BF0F8EFB7F0A0
:106FE8001AC01AF01BC01BF012000A6E000E010135
:106FF8009D6F0DEFB8F0520E096E2B0E086E000E45
:10700800E82EFED7082EFCD7092EFAD700D00101AA
:107018009D2B0A509D5DD8A014EFB8F016EFB8F07C
:10702800FFEFB7F012009F0E0A6EFF0E0B6E200ED8
:1070380008100C6E000E09100D6E0A500C260B502D
:107048000D220D500AE11A0E0C5CD8A02EEFB8F0F4
:1070580031EFB8F0010E32EFB8F0000E086E096A91
:1070680012009F0E0A6EFF0E0B6E08C00CF009C0CE
:107078000DF00A500C260B500D220D500AE11A0E85
:107088000C5CD8A04AEFB8F04DEFB8F0010E4EEF07
:10709800B8F0000E086E096A1200BF0E0A6EFF0EE5
:1070A8000B6E08C00CF009C00DF00A500C260B50EE
:1070B8000D220D500AE11A0E0C5CD8A066EFB8F04C
:1070C80069EFB8F0010E6AEFB8F0000E086E096AB1
:1070D8001200085009100A100B10D8B476EFB8F057
:1070E80078EFB8F080EFB8F0000E081A000E091A11
:1070F800000E0A1A800E0B1A08C008F009C009F021
:107108000AC00AF00BC00BF01200D00E0A6EFF0E78
:107118000B6E08C00CF009C00DF00A500C260B507D
:107128000D220D500AE10A0E0C5CD8A09EEFB8F0B3
:10713800A1EFB8F0010EA2EFB8F0000E086E096AD0
:1071480012003D017995600023F06EFD000E6C6F12
:10715800738B79A5B2EFB8F0B4EFB8F0ADEFB8F033
:1071680074ABB9EFB8F0BCEFB8F0010EBDEFB8F0F2
:10717800000E1200FF0E0816030E09167AA8C7EFB4
:10718800B8F0C9EFB8F0D0EFB8F0060ED8900836CE
:107198000936E82ECAEFB8F00950796E600023F07E
:1071A80078FF1200FF0E0816030E09167EA8DFEFFF
:1071B800B8F0E1EFB8F0E8EFB8F0060ED89008366E
:1071C8000936E82EE2EFB8F009507D6E600023F032
:1071D8007CFF120013C008F014C009F0000E0B6EFB
:1071E800010E0A6E4DECBAF0000E0E6E000E0F6E18
:1071F800000E106E000E116E000E126ED7ECBAF073
:10720800040E120013C008F014C009F0000E0B6E33
:10721800020E0A6E4DECBAF0000E0E6E000E0F6EE6
:10722800000E106E000E116E000E126ED7ECBAF042
:10723800020E120013C008F014C009F0000E0B6E05
:10724800010E0A6E4DECBAF0000E0E6E000E0F6EB7
:10725800000E106E000E116E000E126ED7ECBAF012
:10726800020E120013C008F014C009F0000E0B6ED5
:10727800020E0A6E4DECBAF0000E0E6E000E0F6E86
:10728800000E106E000E116E000E126ED7ECBAF0E2
:10729800040E12003901A3A954EFB9F056EFB9F062
:1072A8004EEFB9F00D0E3D01EA6F3901A3A95FEF6A
:1072B800B9F061EFB9F059EFB9F00A0E3D01EA6F84
:1072C80012003D0173BF6BEFB9F06DEFB9F07BEFC2
:1072D800B9F0000E796F000E7A6F000E766F6C6948
:1072E800510E3A016A6F510E6B6F3D01738F120098
:1072F80001012951FC0B0209296F25052611D8A483
:1073080088EFB9F08AEFB9F08CEFB9F0AFECAFF0D5
:10731800D88001012235B9ECBBF0040E120057F7F2
:107328001CF7B9F7E0F703F8E4F5E0F665F626F59B
:10733800A3F637F88FF7286E756C6C2900010002E8
:0B73480000040008001000008020205E
:10735400000E096E000E086E00F0084A092A09BEE4
:10736400BDEFB9F0095009E1A00E085CD8A0BDEF4B
:10737400B9F0BFEFB9F0AEEFB9F01200010E086E2C
:10738400010129B5C8EFB9F0CAEFB9F0D4EFB9F0EB
:1073940029972269D8ECBBF08FECBAF0B3ECBBF0C0
:1073A40028C108F0085012003BECBAF02FECBBF0F7
:1073B40017ECBBF01BECB5F0ADECBAF0FFECBAF097
:1073C400BBECBAF098ECB7F023ECBBF00BECBBF0E1
:1073D400120008500A026F00CCFF0CF06F00D0FFBF
:1073E4000DF008500B02F3500D2609500A02F35019
:1073F4000D260CC008F00DC009F01200236E22C047
:1074040024F0000E256E240E1D6E000E1E6E000E5E
:10741400206E010E1F6E2350ECECB4F0A00EE82E8B
:10742400FED71200DFECBBF0DCECBBF00009D8B4F3
:107434001EEFBAF020EFBAF026EFBAF0000EBEEC61
:10744400BBF0000EB9ECBBF0000E120016C008F041
:1074540017C009F077ECB5F0085016240C6E0950EB
:1074640017200D6E18C00EF019C00FF086ECB4F0A2
:107474001200000E3901C06F000EC16F000EC26F02
:10748400000EC36F000EC46F000EC56F1D0EC66FD5
:10749400030EC76F1200010129A953EFBAF055EF8B
:1074A400BAF05EEFBAF008C023F109C024F10AC0B3
:1074B40025F10BC026F129991200030E3D017B6FC3
:1074C400040E736F800E746F000E756F000E6C6F78
:1074D4007599200E6E6F7995739F1200086E74EF84
:1074E400BAF000F03901A3A97AEFBAF07CEFBAF050
:1074F40073EFBAF0600023F0EAFD120086EFBAF0F1
:1075040049ECB5F0A4ECB3F0010129B58CEFBAF065
:107514008EEFBAF082EFBAF012003901939393958B
:10752400929F93913D017A917A957A9F7A9D7A936D
:1075340076937695769112006F0060FF07F0010153
:107544007C4B7D2BA08B010EA36F3901A9916000A8
:107554001FF0D8FF1100010EA26E000EA16E000EE6
:10756400A36E9F68000E9E6E3901A791C00EA06E97
:107574001200010EAE6E000EAD6E000EAF6EAB6863
:10758400000EAA6E3901A495C00EAC6E12000EC096
:1075940008F00FC009F010C00AF011C00BF012C0BF
:1075A4000CF0020E34ECB1F012000EC008F00FC063
:1075B40009F010C00AF011C00BF012C00CF0000E5C
:1075C40034ECB1F01200326E2FC02AF03250FAECD3
:1075D400ADF030C028F031C029F0BBECB4F012009B
:1075E400326E2FC02AF03250FAECADF030C028F0E1
:1075F40031C029F07BECB1F012008C0E726E000EDB
:10760400716E000E706E3F015E513F0B80095E6F1C
:1076140012008C0E766E000E756E000E746E3F01B5
:107624005E51CF0B20095E6F12008C0E7A6E000E35
:10763400796E000E786E3F015E51F30B08095E6FA0
:1076440012008C0E7E6E000E7D6E000E7C6E3F016D
:107654005E51FC0B01095E6F1200600E3901D96F97
:10766400000EDB6F000EDD6F080EDF6F000EDE6FA5
:10767400120001012951FC0B0209296F2251222514
:10768400B9ECBBF0030E12003D0178BB4CEFBBF02C
:107694004FEFBBF0010E50EFBBF0000E12003D01A6
:1076A40074BB57EFBBF05AEFBBF0010E5BEFBBF0BE
:1076B400000E12003D0178B162EFBBF065EFBBF044
:1076C400010E66EFBBF0000E12003D0179B56DEFBF
:1076D400BBF070EFBBF0010E71EFBBF0000E1200B7
:1076E4003D0176B978EFBBF07BEFBBF0010E7CEF88
:1076F400BBF0000E12003D0179BF83EFBBF086EFB3
:10770400BBF0010E87EFBBF0000E1200C3ECBBF020
:1077140001012995020E286F0F0E1200C3ECBBF075
:1077240001012995000E286F0F0E120008C0EBF11D
:1077340009C0ECF10AC0EDF11200E2ECBBF0DFECA1
:10774400BBF0ADECBBF0120001012551BEECBBF067
:107754007CECB9F0120001012995000E286F0F0E80
:1077640012003D01739F000E796F78851200086E38
:10777400600023F06BFD1200086E600023F06CFDC6
:1077840012003D01739F7885738F1200000E4DEC3B
:10779400B6F01200E2ECBBF0090E1200E5ECBBF00F
:1077A400040E1200E5ECBBF0030E1200000E3D01C6
:1077B400796F12003D016C5112003D01739B120060
:1077C4003D01748D12003D01749D12003D016A510A
:1077D40012003D01738D12003D01739D12003D01A5
:1077E400799512003D01769912003D01799F1200AE
:1077F400010E1200020E1200050E1200010E1200FC
:08780400140012001100120033
:020000040020DA
:10000000FFFFFFFFFFFFFFFFFFFFFFFFFFFFFFFF00
:020000040030CA
:0A0000008CFFFFFF9FFFFFFFFFFFD3
:00000001FF
